:040000000C94BA01A1
:080024000C94C6020C94950235
:040040000C944007D5
:040048000C945E2195
:040078000C94391893
:14008C00C023C523CA23CF23D423D923DE23E323E823ED23A1
:1400A000F223F723FC23012406240B24102415241A241F2492
:1400B400242429242E2433241725382446254B255025552598
:1400C8005A255F25642569256E25732578257D25822587254D
:1400DC008C2591254C2696257B26802685268A268F2694266B
:1400F00099269E26A326A826AD26B226B726BC26C126C626A5
:140104003327CB26CF2DD72DDF2DE72DEF2DF72DFF2D072EDB
:140118000F2E172E1F2E272E2F2E372E3F2E472E4F2E572E09
:14012C005F2E672E6B2E6F2E732E772E7B2ED12ED52EDD2E6B
:14014000E52EED2EF52EFA2EFF2E042F092F112F192F212FC2
:14015400292F312F392F3D2FA830AD30B230B730C430C930A0
:14016800CE30D330D830DD30E230E730EC30F130F630FB30B6
:14017C000031053110312C313E314231463156316A316F314F
:140190007331613478349034A734BA34CE348235823527351D
:1401A4002B3582358235823582358235823582358235823578
:1401B8008235533557356B354F35F53482354B35E134433557
:1401CC008235EB343F3582358235823582358235473524475B
:1401E00050524D432C00000302050003050104060204010089
:1401F4000100D00700000000000000001F003B005A007800F3
:140208009700B500D400F300110130014E016D0100FFFFFFD2
:14021C00FFFF000020203F0020204A5441470020205761747F
:140230006368646F6700202042726F776E2D6F7574002020A8
:1402440045787465726E616C002020506F776572204F4E0059
:1402580020200052657365742044617465202F2054696D65B3
:14026C00202020202020205265736574205479706500436F27
:140280006D6D756E69636174696F6E20746F20475053206435
:140294006576696365206661696C656400453300436F7272B7
:1402A800656374656420746F206C6F63616C2074696D653A06
:1402BC0020200054696D653A2020004461746520284D2F445F
:1402D0002F59293A2020005554432028477265656E77696387
:1402E40068292044617465202F2054696D653A00285365655A
:1402F8002048656C7020666F722073746174757320636F64C8
:14030C006573290047505320436F6D6D756E69636174696FEA
:140320006E205374617475733A20004D4355435352005275C9
:140334006E6E696E6700562B204C4F5700562B204F4B004984
:140348004E4954003031323334353637383961626364656654
:14035C006768696A6B6C6D6E6F707172737475767778797AC3
:0303700000010089
:14037400CFEFD0E1CDBFDEBFC051D0400AEA08830024EBE747
:14038800F2E014E0E13FF10711F00192FBCF0083E8EFF1E0FA
:14039C00A0E0B1E013E0E337F10721F0C89531960D92F9CF9B
:1403B0000E94070AFFCF0E94AB3D002321F4599A83E089B95E
:1403C40011C0013021F4599885E089B90BC0023021F4599873
:1403D80087E089B905C0033019F4599887E189B986E080934F
:1403EC00950088E98AB9ACB078940E94993D08952CB02092A9
:140400007B0208955D9BFECF0CB908950E94AE3D6801AA24E3
:14041400BB240AC0F60100810E946C3EC50101965C01C601E6
:1404280001966C01F6012080222091F7A89501E010E00E94AB
:14043C00A53D089508950E94AB3D87B1806C87B927B027B8EC
:14045000329A379A85B7806185BF85B7806485BF88950027F2
:1404640022D05801379885B78F7B85BF0E94993D089587B193
:14047800806C87B927B0202A27B886B1856086B9379A08957B
:14048C0037980895379A369A089504B1112725B03324322C3B
:1404A0002224020D131D349A08950E94AB3D379A27B0202ADC
:1404B40027B8369A3699FECFA4B0BB2425B03324322C2224E6
:1404C800A20CB31C85010E94993D0895222420929A002092C4
:1404DC009B0086E080939D008FEB809399002092980088E97A
:1404F00080939A000895222420929A00089588E980939A0061
:14050400089500919C000895222425BC87B78F7387BF8DE45E
:1405180084BD83EB83BD87B7806487BF85E085BD08958A9317
:14052C009A938FB78A938DE484BD809181028F5F8093810261
:14054000809180028F5F8093800280917F028F5F80937F027D
:1405540080917E028F5F80937E0289918FBF99918991189528
:14056800222425BC87B78F7387BF88E384BD88EC83BD87B734
:14057C00806887BF8CE085BD0895222424BC08958A939A93E5
:140590008FB78A9380917E028F5F80937E02809181028F5F60
:1405A4008093810289918FBF999189911895889A899A909AE5
:1405B800919A0895909A919A899A91980895899A91989098B5
:1405CC00909A919A0895909A0000909808950E94AE3DC02EBF
:1405E000899A9098AA240BC08C2D8078803811F4919A01C0C9
:1405F4009198909ACC0C9098A3948A2D883090F31CD0002368
:14060800E9F70E94A53D08950E94AE3DCC24AA240AC0CC0CF0
:14061C008998909A819B03C08C2D8160C82E9098A3948A2DFA
:14063000883098F3CEDF0C2D0E94A53D0895002790988998FC
:14064400909A819B01C001E0909808950E94AE3DA22EC02EAA
:1406580090988C2D8870883011F4919A01C09198B4DF8C2D97
:14066C008470843011F4919A01C09198ACDF8C2D82708230D0
:1406800011F4919A01C09198A4DF8C2D8170813011F4919A3E
:1406940001C091989CDF8A2D8470843011F4919A01C0919874
:1406A80094DF8A2D8270823011F4919A01C091988CDF8A2D34
:1406BC008170813011F4919A01C0919884DF0C80002011F05E
:1406D000919A01C091987DDFB2DF0023E9F70E94A53D0895F0
:1406E4000E94B23DA22EE02E2197CF80D88464DF22242882FD
:1406F8002E2D0AE0A9DF0A2D6CDF00276ADF80E091E05C0101
:14070C0007C0F60101916F0162DFC50101975C01AA20B9F7A3
:14072000BB20A9F750DF21960E94A83D08950E94AE3D590159
:14073400C02E219741DF222428822C2D0AE086DF8501012F9D
:14074800112747DF0A2D107044DF0D8142DF37DF21960E9447
:14075C00A53D08950E94AE3D6901A02E219728DF2224288296
:140770002A2D0AE06DDF8601012F11272EDF0C2D10702BDF29
:140784001BDF81E088832A2D0AE060DF3FDFA02E18DF0A2D61
:1407980021960E94A53D08950027112702C00F5F1F4F003741
:1407AC00E7E11E07D0F308950E94AE3DA02EA895C0900401FF
:1407C000DD24CC2011F4DD20B9F0C6018130E0E09E0709F4B3
:1407D40030C08230E0E09E0709F44DC08030E0E09E070CF4EB
:1407E8007EC0C6018930E0E09E0709F456C077C08EED91E0A4
:1407FC00E0910301FF27E80FF91FE491AE1631F480910301CC
:140810008F5F8093030103C022242092030180910301873044
:1408240009F0F8C081E080930401222420920501F1C08A2D30
:140838008C3289F48CE992E0E0910501FF27E80FF91F222498
:14084C00208220920501809104018F5F80930401DDC08CE910
:1408600092E0E0910501FF27E80FF91FA082809105018F5F3F
:1408740080930501CFC08A2D8C3249F4222420920501809107
:1408880004018F5F80930401C3C0A0929402809105018F5F01
:14089C0080930501BBC08A2D8C3289F485E992E0E09105016B
:1408B000FF27E80FF91F2224208220920501809104018F5F5B
:1408C40080930401A7C085E992E0E0910501FF27E80FF91F15
:1408D800A082809105018F5F8093050199C08A2D8C3229F4E1
:1408EC00809104018F5F809304018A2D8A3009F08DC02224DF
:140900002092040120920301AA243DC02A2C3324220C331C81
:140914008CE992E0F101E80FF91F40808AE0849DC001805EFD
:140928009140EDE9F2E0D101AE0FBF1F9C919053890FE1E963
:14093C00F2E0AA2DBB27AE0FBF1F8C932A2C3324220C331C38
:1409500085E992E0F101E80FF91F40808AE0849DC001805EC8
:140964009140E6E9F2E0D101AE0FBF1F9C919053890FEEE822
:14097800F2E0AA2DBB27AE0FBF1F8C93A3948A2D833008F489
:14098C00BFCF82E892E0E8E8F2E006E010E0FA93EA939A933E
:1409A0008A930E94543E209091022092820220909202209283
:1409B4008302209093022092840220908E0220928502209004
:1409C8008F022092860220909002209287021CE300918A02B7
:1409DC000F5F0E94413D20908402201631F4809101018F5FE7
:1409F0008093010105C0222420920101209202018091010157
:140A0400843041F481E0809302018091010181508093010185
:140A18000E94A53D08950E94B23DC22E580129972224332472
:140A2C003092A6022092A502A89524E039E000270E94B0031D
:140A4000202E3324322C22243C822B8225E039E000270E9407
:140A5400B003202E33240B801C80020C131C1C820B820F8414
:140A680008822C2D85010E9420091E830D8320E039E00027D5
:140A7C000E94B003202E332438862F8221E039E000270E941A
:140A9000B003A02EBB2422E039E000270E94B003E02ECE2C53
:140AA400DD24DC2CCC2423E039E000270E94B003E02E2E2C45
:140AB8003324C20CD31C2F80388428822A2D86010E94200958
:140ACC0068012D803E80201A310A3A8229822B813C8181017B
:140AE0003AD129960E94A83D08950E94AE3DC02E2090F304F2
:140AF4008CE3829D50012090F2043324A20CB31CA895CC206C
:140B080009F46DC022243092A6022092A502910104E010E040
:140B1C000E94593DF80184ED92E0E80FF91F208031802A1413
:140B30003B0408F058C036C02091A5023091A60204E010E0D7
:140B44000E94593D84ED92E0F801E80FF91F2080318088EDB4
:140B580092E0F801E80FF91F408051804214530408F425C0F0
:140B6C002091A5023091A60204E010E00E94593DF80188ED3A
:140B800092E0E80FF91F20803180A214B30408F412C0809143
:140B9400A5029091A60201969093A6028093A5028091A50209
:140BA8009091A6028F30E0E09E070CF4C1CF2091A5023091A3
:140BBC00A60204E010E00E94593DF80186ED92E0E80FF91F84
:140BD00000813BD08091A5029091A60201969093A60280938F
:140BE400A5028091A5029091A6028031E0E09E073CF59C01F1
:140BF80004E010E00E94593DF80184ED92E0E80FF91F208052
:140C0C003180A214B304C1F42091A5023091A60204E010E06C
:140C20000E94593DF80186ED92E0E80FF91F00810CD080912D
:140C3400A5029091A60201969093A6028093A5020E94A53D9C
:140C480008950E94AB3DA02E80E38A9DC001885E9E4F5C0128
:140C5C00A8959C0100270E94B0030093AF0395012F5F3F4F37
:140C700000270E94B0030093AE0395012D5F3F4F00270E9437
:140C8400B0030093CF03202E87E6829D800100571E4F24E61B
:140C980030E00E949A3C0093CE032090CF038EE6829D8001C6
:140CAC0006571D4F24E630E00E949A3C0093CD0395012C5F55
:140CC0003F4F00270E94B0030093650395012B5F3F4F002746
:140CD4000E94B0030093D70395012A5F3F4F00270E94B00321
:140CE8000093AD039501295F3F4F00270E94B0030093AC034B
:140CFC009501285F3F4F00270E94B0030093B0039501265F5C
:140D10003F4F00270E94B0030093700381E080933603809101
:140D2400E303813011F0833069F42090AF03222021F42090AA
:140D3800B003222029F01A9A81E08093350304C01A9822247D
:140D4C00209235030E94993D08950E94B23D59016801229787
:140D6000A895C6018030E0E09E073CF0A816B90624F0AA20DF
:140D740081F4BB2071F48091F70499278C5F964F5C018091AC
:140D8800F704813041F4C50107965C0104C0C601835F964F64
:140D9C005C01950100270E94B003A02E80E58A9DC001885ED3
:140DB0009B4F99838883CC24DD243EC003E010E096010E9423
:140DC400593DE880F980E00EF11E970100270E94B003A02EC5
:140DD800BB24BA2CAA2497012F5F3F4F00270E94B003202EF6
:140DEC003324A20CB31C04E010E096010E94593DF80184ED12
:140E000092E0E80FF91FB182A08297012E5F3F4F00270E948C
:140E1400B003202E04E010E096010E94593DF80186ED92E048
:140E2800E80FF91F332431822082C60101966C018FE090E051
:140E3C008C159D0508F0BCCF22960E94A83D0895F89483B73A
:140E50008F7B83BF83B7877F83BF83B78D7F83BF83B7856019
:140E640083BF87B78C7F87BF80B7886080BF222422BE87B7E7
:140E7800816087BF789408952A928A939A932FB62A928091DE
:140E8C002A0390912B03019690932B0380932A038091B002EB
:140EA0008F5F8093B00281E080937C03809368038091F10414
:140EB4008F5F282E2092F1048BE3821530F422242092F10429
:140EC80081E08093AF0229902FBE9991899129901895809190
:140EDC00F2048F5F282E2092F2048C3309F0CCC022242092E4
:140EF000F20481E080937B038091F3048F5F282E2092F30411
:140F0400883109F062C022242092F3042092A70281E0809347
:140F1800AE028091F4048F5F282E2092F404803249F480911E
:140F2C00F5048F5F8093F50481E08093F40439C08091F40450
:140F40008F3199F48091F504843031F0863021F0893011F0F0
:140F54008B3059F58091F5048F5F8093F50481E08093F40410
:140F680022C08091F4048E3159F48091F5048230D1F48F5F0F
:140F7C008093F50481E08093F40413C08091F4048D3179F4E2
:140F90008091F504823059F476D0002341F08091F5048F5FB2
:140FA4008093F50481E08093F4048091F5048D3041F481E064
:140FB8008093F5048091F6048F5F8093F60476D00093F7043F
:140FCC005BC08091F304853089F480E19EE090932D03809377
:140FE0002C032224332430922B0320922A032090E20320921B
:140FF400AD0246C08091F304823009F041C08091F5048330C3
:14100800D9F487E02090F4048215B0F4822D8F3098F48091B2
:14101C00F704813079F481E08093AC022FE130E000270E949C
:14103000B003013029F48091F3048F5F8093F3048091F504A1
:141044008B30F1F48091F4048830D0F48091F7048130B1F411
:1410580022242092AC022FE130E000270E94B003002361F0CE
:14106C002090A702222041F48091F30481508093F30481E05C
:141080008093A702089514E60091F6040E94413D002341F406
:1410940020E931E00091F60411270E94963C07C024E030E01C
:1410A8000091F60411270E94963C08950E94AE3D2C9786EE9C
:1410BC0091E0FE010CE010E0FA93EA939A938A930E943B3E65
:1410D0008091F60499278053984F9093AA028093A9028091E9
:1410E400F60499278053984F5C018091F504833020F481E0F5
:1410F80090E06C0102C0CC24DD24AC18BD0824E030E0850131
:14110C000E949A3C1501200E311E24E630E085010E949A3CAC
:14112000201A310A20E931E085010E949A3C200E311ECE01E2
:141134000197E091F504FF27E80FF91F40805524240C351CB6
:141148004090F4045524240C351C27E030E081010E94963CC4
:14115C000F5F1F4F2C960E94A53D08952FE130E000270E94D7
:14117000B003002309F462C09DDF0093F7042FE130E0002725
:141184000E94B003002309F454C08091F504833009F5809102
:14119800F404883020F422242092AC0248C087E02090F404C2
:1411AC00821580F4822D8F3068F487502090F704821520F031
:1411C00081E08093AC0237C022242092AC0233C081E08093F5
:1411D400AC022FC083E02090F504821538F4822D8B3020F41D
:1411E80081E08093AC0223C08091F5048B30A1F48091F4048B
:1411FC00883060F43090F704831520F022242092AC0213C0F7
:1412100081E08093AC020FC022242092AC020BC08AE020904E
:14122400F504821518F0822D843018F422242092AC02009178
:14123800AC0201C0002708950E94B23DAA24BB24C801805D8B
:14124C009740837090708030890721F481E090E06C0102C06F
:14126000CC24DD24EC2C16C0C801805D97408370907080307B
:14127400890721F481E090E06C0102C0CC24DD2420901E0101
:1412880030901F012C0C3D1CA20CB31C18010150104080ED3D
:14129C0097E08215930510F382E0821730F4EE2021F081E0F6
:1412B00090E06C0102C0CC24DD2482E0829FF00184E091E051
:1412C400E80FF91F208031802C0C3D1CA20CB31C2E803324A3
:1412D800A20CB31C85010E94A83D08953A932A930E94B23DC0
:1412EC003801269782EF91E0FE0106E010E0FA93EA939A930A
:141300008A930E943B3E8EE691E04C01EE24E394AA2422C036
:141314000C841D84081819081D860C868C819D8101969D833C
:141328008C83805D9740837090708030890721F481E090E0D5
:14133C006C0102C0CC24DD24EC2C2E2C332440901E015090E5
:141350001F01420C531C42010C841D8480149104C8F28CE0E9
:14136400A82E3DC082E08A1530F4EE2021F081E090E06C0120
:1413780002C0CC24DD2482E08A9DF00184E091E0E80FF91F50
:14138C00208031802C0C3D1C0C841D842014310408F582E072
:1413A0008A1530F4EE2021F081E090E06C0102C0CC24DD2466
:1413B40082E08A9DF00184E091E0E80FF91F208031802C0C3E
:1413C8003D1C0C841D84021813081D860C862A2C33243B82B3
:1413DC002A8205C0AA9422242A1408F4BFCF0C841D84198274
:1413F0000882CE0106E010E07A926A929A938A930E94543E34
:1414040026960E94A83D2296089521978BEE81BB00E40E9449
:141418001A3C00E40E941A3C00E40E941A3CF89484B7806803
:14142C0084BF84B7806884BF66270E94260705E00E943B02E3
:14144000789400EA16E821E030E00E94323C05E00E945502A5
:141454008BE992E08017910734F422242092A8030E94F11FF2
:1414680012C000EA16E821E030E00E94323C81E080937903A5
:14147C000E94AC2080916200877F809362000E94CD20F894E5
:141490000E9486020E9430210E94D90278940E94B716069994
:1414A4001CC1C19A81E08093AF03199886B3827086958093CC
:1414B800A6032224332430922B0320922A037EC0A8952090E0
:1414CC0081022220A1F020908403222039F000E20E94D71E9B
:1414E00022242092840306C000E20E94C31E81E08093840353
:1414F400222420928102B19904C081E090E05C0102C0AA249D
:14150800BB242090A6033324250142205320442019F455205F
:14151C0009F452C005E00E9455021801442437FC40945524CD
:1415300047FC50943092CD022092CC025092CF024092CE021A
:1415440080E991E4AFE1B0E05A924A923A922A928C019D011A
:141558000E94D03C1093D1020093D0023093D3022093D202D7
:14156C00180130921B0320921A0320901A0330901B03232CA9
:14158000332428822AE230E000270E9497030E94D0032090B2
:141594001A0330901B0328822BE230E000270E9497030E947C
:1415A800D003A89500E80E941A3C00E80E941A3C8AE090E085
:1415BC0090932B0380932A0380912A0390912B038530E0E088
:1415D0009E0708F479CF0E94F51B05E00E945502180144240D
:1415E40037FC4094552447FC50943092CD022092CC02509259
:1415F800CF024092CE0220901A0330901B03442455248090D0
:14160C00CE029090CF026090CC027090CD025A924A923A92E8
:141620002A92830194010E94693D86E090E0A0E0B0E03A93E6
:141634002A931A930A938C019D010E94693D1801290180E085
:1416480094E1A0E0B0E0280E391E4A1E5B1E80E098E2A0E041
:14165C00B0E0BA93AA939A938A93810192010E94D03C1093B0
:14167000D1020093D0023093D3022093D20284E690E0A0E0B5
:14168400B0E0BA93AA939A938A930E94D03C0E946815A895E4
:1416980000EA16E821E030E00E94323C0091D0021091D1025E
:1416AC000E946815A89500EA16E821E030E00E94323C00279E
:1416C00011270E9468150AC0A895B19903C00E94D21504C05E
:1416D4000CEB10E00E946815F5CFF8942CE230E000270E94C5
:1416E800B00300938403023018F40E94DB0103C000270E94D9
:1416FC00DB0178940FE412E00E9406020DE00E9402022FE1C0
:1417100030E000270E94B00381E0801740F488832FE130E0E2
:1417240000270E9497030E94D0030E94EB1E8FEF9FEFAFEF84
:14173800B0E04090CA025090CB022090C8023090C902281681
:14174C0039064A065B0649F08FEF9FEFA3E0B0E08215930512
:14176000A405B50588F58FEF88832BE130E000270E9497038D
:141774000E94D00380E09CE0A0E0B0E09093C9028093C80235
:14178800B093CB02A093CA022224288228E130E000270E946C
:14179C0097030E94D0038CE0888329E130E000270E94970336
:1417B0000E94D00380E09CE088832AE130E000270E9497034B
:1417C4000E94D00381E080937C028FEF80937B028093210167
:1417D800809322018093230180932401809325012BE130E003
:1417EC0000270E94B003009384030F3FF9F422242092840399
:1418000028822BE130E000270E9497030E94D00320908403FF
:1418140028822CE130E000270E9497030E94D00320908403EA
:1418280028822DE130E000270E9497030E94D0030E94721FD9
:14183C0028E230E000270E94B0030093840324E630E08A0143
:141850000E94B63C2090840333242016310681F024E630E06A
:141864008A010E94B63C00938403202E288228E230E00027FE
:141878000E9497030E94D00329E230E000270E94B003009381
:14188C00840324E630E08A010E94B63C980104E610E00E9473
:1418A000593D1A01201A310A40908403552442145304B9F0E8
:1418B40024E630E08A010E94B63C980104E610E00E94593D3C
:1418C8001A01201A310A20928403288229E230E000270E94B5
:1418DC0097030E94D00322242092840333C080918403883126
:1418F000C1F42224209284030FC0222428822091840333275F
:1419040000270E9497030E94D003809184038F5F80938403D7
:1419180080918403883168F31BC020918403332700270E94D9
:14192C00B003202E332430921D0320921C03C1018F3FE0E04C
:141940009E0709F009C0809184038F5F809384038091840374
:14195400893148F20E94F51B05E00E94550220901803309070
:1419680019032016310678F409E412E00E9406020DE00E945E
:14197C00020281E08093A8030E94F11F0E94200213C002E405
:1419900012E00E9406020DE00E94020281E0809379030E9482
:1419A400AC2080916200877F809362000E94CD202DE230E0C7
:1419B80000270E94B0030F3F09F0A7C18EE4888322273327D0
:1419CC0000270E9497030E94D00385E6888321E030E0002781
:1419E0000E9497030E94D00387E7888322E030E000270E94EE
:1419F40097030E94D00389E1888320E230E000270E949703E6
:141A08000E94D0032224288221E230E000270E9497030E944D
:141A1C00D00381E088832FE130E000270E9497030E94D0037F
:141A300081E0888326E230E000270E9497030E94D00381E0E5
:141A4400888327E230E000270E9497030E94D00381E0888326
:141A58002DE230E000270E9497030E94D00381E088832EE207
:141A6C0030E000270E9497030E94D00389E188832FE230E0E8
:141A800000270E9497030E94D00383E2888320E330E00027D0
:141A94000E9497030E94D0038AE1888321E330E000270E943A
:141AA80097030E94D00384E2888322E330E000270E94970332
:141ABC000E94D00381E0888323E330E000270E9497030E941A
:141AD000D0038DE2888324E330E000270E9497030E94D003C6
:141AE40087E3888325E330E000270E9497030E94D00381E028
:141AF800888327E330E000270E9497030E94D00381E0888371
:141B0C0028E330E000270E9497030E94D00381E0888329E35A
:141B200030E000270E9497030E94D003222428822AE330E0BC
:141B340000270E9497030E94D00381E088832BE330E0002714
:141B48000E9497030E94D00381E088832CE330E000270E9484
:141B5C0097030E94D00387EC88832DE330E000270E94970365
:141B70000E94D00387EC88832EE330E000270E9497030E9448
:141B8400D003222428822FE330E000270E9497030E94D00390
:141B98002224288220E430E000270E9497030E94D00382E0FB
:141BAC00888321E430E000270E9497030E94D00388E18883B9
:141BC00022E430E000270E9497030E94D00387EC888325E49C
:141BD40030E000270E9497030E94D00387EC888326E430E07D
:141BE80000270E9497030E94D0032224288227E430E00027DF
:141BFC000E9497030E94D0032224288228E430E000270E944F
:141C100097030E94D00387EC888329E430E000270E949703B3
:141C24000E94D00387EC88832AE430E000270E9497030E9496
:141C3800D003222428822BE430E000270E9497030E94D003DE
:141C4C0081E088832CE430E000270E9497030E94D00385E0BB
:141C600088832DE430E000270E9497030E94D003222428827C
:141C74002EE430E000270E9497030E94D003222428822FE45F
:141C880030E000270E9497030E94D0032224288220E530E05B
:141C9C0000270E9497030E94D0032224288221E530E000272F
:141CB0000E9497030E94D00381E0888322E530E000270E9423
:141CC40097030E94D00381E0888323E530E000270E94970316
:141CD8000E94D00381E0888324E530E000270E9497030E94F9
:141CEC00D00381E0888325E530E000270E9497030E94D003B3
:141D00002224288220E630E000270E9497030E94D0030E944F
:141D1400E01CF8940E944E2178940AE312E00E9406020DE0A0
:141D28000E94020204EF0E94020287E12090F304821578F05A
:141D3C008BE32090F204821550F08FE12090F404821528F0E1
:141D50008CE02090F504821570F422242092F1042092F204DA
:141D64002092F30481E08093F6048093F5048093F4042224F7
:141D780084B78F71281608F070C020E630E000270E94B00324
:141D8C00009384032090F4042882202E86E0829D90012F59EB
:141DA0003F4F00270E9497030E94D0032090F50428822090C6
:141DB400840386E0829D90012E593F4F00270E9497030E9464
:141DC800D0032090F60428822090840386E0829D90012D590D
:141DDC003F4F00270E9497030E94D0032090F304288220908C
:141DF000840386E0829D90012C593F4F00270E9497030E942A
:141E0400D0032090F20428822090840386E0829D90012B59D6
:141E18003F4F00270E9497030E94D00324B628822090840395
:141E2C0086E0829D90012A593F4F00270E9497030E94D003A3
:141E40001AE0009184030F5F0E94413D00938403202E2882DC
:141E540020E630E000270E9497030E94D00303E312E00E9412
:141E6800060204B70E94020280E884BF6CC28AE02090B00258
:141E7C00821598F422242092B00280912001807F8093200120
:141E90002092880320927F03332430922903209228032092F9
:141EA4008303222430906803231418F4A895209268032090E6
:141EB800AF02222009F485C020905C0330905D03222019F463
:141ECC00332009F470C08091F204853009F06BC02224332405
:141EE00030925D0320925C038091F704813009F060C020E2E3
:141EF40030E000270E94B0032224201608F057C021E230E0B0
:141F080000270E94B003013049F520E230E000270E94B0034C
:141F1C00009384032CE330E011270E94963C10931F03009374
:141F30001E031CE3009184030E94433D00938403802F8F5F8C
:141F44002090F204281A2092F20420901E0330901F038CE3D7
:141F580090E0821993098093F10427C020E230E000270E9404
:141F6C00B003009384032CE330E011270E94963C10931F0304
:141F800000931E031CE3009184030E94433D00938403309086
:141F9400F204300E3092F20420901E0330901F034090F104D5
:141FA8005524420C531C4092F10481E08093B5020E946D07E7
:141FBC00A89522242092AF0281E0809336032090E4032220A5
:141FD00029F12090B5022220F1F12090AE022220A1F081E0C4
:141FE40090E090935D0380935C032090F40428822091F50488
:141FF8000091A9021091AA020E940F0522242092AE020027C7
:14200C000E9475050093840322242092B5021DC02090AE029E
:14202000222049F081E090E090935D0380935C032224209273
:14203400AE022090D00380B3807182958F70821541F080B330
:14204800807182958F708093D0030E94E01C8091AD02813088
:14205C00A9F42EE430E000270E94B0032224201668F42FE04E
:1420700030E000912A0310912B030E94B43C0030010711F4F0
:142084000E9445188091E303823069F480913603813009F04F
:142098005FC00091AE03112717D522242092360357C02090B7
:1420AC00CB0330907E02231440F480917D028F5F80937D0297
:1420C000222420927E0220907003332440902203509023031F
:1420D4004214530484F120906F03222061F120903803309075
:1420E8007D02231418F4222420927D022090370330907D0282
:1420FC00231498F42090CC0330907E02231410F445D524C015
:142110002090C803222011F445D51EC00091C8031127D6D4C3
:1421240019C02090CC0330907E02231410F432D511C036D5F1
:142138000FC0222420927D022090CC0330907E02231410F453
:14214C0025D504C00091C8031127BCD420905703222021F040
:142160008091AD03873C21F404EB0E94D71E33C020903B036B
:14217400222021F42090AD03222029F580915703813021F40F
:1421880004EB0E94C31E23C02090770330908002231450F407
:14219C0022242092800204EB0E94C31E81E08093640313C095
:1421B0002090780330908002231468F404EB0E94D71E22244F
:1421C4002092640306C004EB0E94D71E222420926403209093
:1421D8003C03222009F47AC020903A03222029F42090AC0390
:1421EC00222009F06EC080915603813021F405EB0E94C31ED3
:1422000069C02090570330905603321421F480913B03813023
:1422140029F02090AD03222009F03AC080915603833079F47E
:1422280080915503815020906403282621F005EB0E94C31E7F
:14223C004BC005EB0E94D71E47C082E080935603882309F47F
:1422500041C020908002222021F480915503813041F0809194
:1422640080028B3059F480915503823039F4222420927F021B
:1422780005EB0E94C31E2AC02090760330907F02231420F53F
:14228C0005EB0E94D71E20C080915603823011F08330D1F442
:1422A0002090750330907F02231438F4222420927F0205EBF5
:1422B4000E94C31E0DC02090760330907F02231438F405EB09
:1422C8000E94D71E03C005EB0E94D71E809135038130F1F442
:1422DC0020908103222011F037D018C084E02090810282156A
:1422F00098F42224209281032092CA032092C80384E180935E
:14230400CC038AE08093CB0300271127DFD32224209281021F
:142318000E944220222420927D0320907B03222039F0222456
:14232C0020927B030E941A3B0E946C3B20908703222031F090
:14234000A8950E94E5352224209287030BD693CD2196089579
:142354000E94AB3D222420928102209281032DE230E00027F4
:142368000E94B003073C09F05CC081E080936503A8952090EB
:14237C0086032220E9F422242092CA0380EA809386030E9438
:14239000E43E98012F71307004E610E00E94593DC801885388
:1423A4009F4F909327038093260324E630E08C010E94B63C73
:1423B8000093800380918603815080938603843600F515E050
:1423CC00082F0E94433D20908003209E80012AE030E00E9476
:1423E0009A3C2090260330902703201A310A3092270320923D
:1423F400260324E630E081010E94B63CC80147968093CA03F6
:1424080010C0809186038C3860F424E630E0009126031091C9
:14241C0027030E94B63CC80147968093CA0322243090CA0395
:14243000231438F4232C2092630388E0809362030DC02224DB
:1424440030906203231428F4832D81508093620303C022240A
:142458002092630320907203222041F0209063033324309291
:14246C0021032092200307C02090CA03332430922103209230
:14248000200380916E038F5F80936E0318E0082F0E94413DE2
:1424940000936E03209020033090210388ED93E0E02FFF275C
:1424A800E80FF91F208220926C032092580382E080936B035E
:1424BC0081E080936A0320906E032092690380938403B2C0E0
:1424D00020906903222019F488E08093690380916903815058
:1424E4008093690388ED93E0E0916903FF27E80FF91F2080CB
:1424F80020926103E0916903FF27E80FF91F2080332432146B
:14250C0008F088C020905803222041F4E0916903FF27E80FFF
:14252000F91F20802092580388ED93E0E0916903FF27E80F00
:14253400F91F208030906C03231431F480916A038F5F8093D1
:142548006A0360C088ED93E0E0916903FF27E80FF91F208058
:14255C0030906C03321420F481E08093660303C0222420924A
:14257000660388ED93E0E0916903FF27E80FF91F20802092A2
:142584005E0320906C03332400915E031127021913090E9469
:14259800823C81E090E08017910784F480936A0382E0809304
:1425AC006B0388ED93E0E0916903FF27E80FF91F2080209261
:1425C000580324C080916B03823051F42090660320926B0319
:1425D40080916A038F5F80936A0316C02090660380916B0399
:1425E800820D813051F482E080936A0320926B0320906C0339
:1425FC002092580305C080916A038F5F80936A0388ED93E025
:14261000E0916903FF27E80FF91F208020926C0380916A0365
:14262400853009F40AC0809184038F5F80938403809184036E
:14263800883008F449CF80916A03853050F020905803209292
:14264C0060032092730386E080935F0324C0222420926003D5
:142660002090220330902303009120031091210302191309FB
:142674000E94823C0230E0E01E0724F486E080935F030DC01B
:1426880081E020905F03821528F4822D815080935F0303C060
:14269C0022242092730380913903823000F52224309073034C
:1426B000231490F420905903321451F088E080933903232CC2
:1426C4003324309223032092220312C081E0809339030EC09C
:1426D8002224209239033324309223032092220305C08091CE
:1426EC003903815080933903209024033090250340902203CA
:14270000509023034218530881E090E08415950514F45C01A1
:1427140002C0AA24BB24209124033091250385010E94593DC3
:1427280000300107F1F42090220330902303409024035090EE
:14273C0025034218530882E090E0841595051CF481E05C01D9
:1427500002C0AA24BB24209124033091250385010E94593D87
:142764000030010721F0009124030E94BC392090390322209B
:1427780019F0822D883011F520905A032220C1F020907103B3
:14278C00332440902203509023034214530439F42090240336
:1427A000309025032092C8030DC02090220330902303209286
:1427B400C80306C020902203309023032092C8032224309042
:1427C8005A03231428F4832D815080935A031CC02224209288
:1427DC0071032090220330902303009124031091250302191E
:1427F00013090E94823C0130E0E01E0749F48FE080935A0327
:14280400209024033090250320927103209022033090230320
:1428180030922503209224032090CF0333244090220350903B
:14282C00230342145304B4F181E08093B1032090CE03332420
:142840004214530404F12090CD033324421453046CF082E0A0
:142854008093CC0385E08093CB0384E08093370389E080931B
:14286800380320C083E08093CC0387E08093CB0384E080933D
:14287C00370388E08093380313C086E08093CC038AE08093C0
:14289000CB0383E08093370386E08093380306C084E18093C4
:1428A400CC038AE08093CB032090AD0333244090220350907A
:1428B800230342145304C4F081E080933B03809157038330B5
:1428CC00A1F42090B1033090CC03329C009278033090CB0307
:1428E000329C0092770320907E022092800203C022242092EB
:1428F4003B032090AC03332440902203509023034214530434
:14290800C4F081E080933A03809156038330A1F42090B10340
:14291C003090CC03329C009276033090CB03329C00927503D9
:1429300020907E0220927F0203C0222420923A032090D703AE
:14294400332440902203509023034214530494F08091D60312
:14295800813031F422242092C8032092C90308C08091D603A2
:14296C00823021F42090AE032092C803209065033324409073
:14298000220350902303421453041CF422242092C803809187
:14299400E303833021F42090AE032092C8030E94993D08958E
:1429A8000E94B23DC22EE02EAE8085EB93E0EE2DFF27E80F43
:1429BC00F91F20802092B303EC2DFF27E80FF91F2080209247
:1429D000B20380916200806880936200DF9A2090B30325BAB0
:1429E4002090B2032BBA22242092810201C0A89520908102E9
:1429F8002A14D8F32224209281020027112764D00E94A83D2D
:142A0C0008950E94AE3DA22EC02EA89514E60C2D0E94433D3C
:142A20000093840385EB93E0E02FFF27E80FF91F208020920F
:142A3400B403202E8AE0829D10012AE030E00C2D11270E94C2
:142A48009A3C28014218530850921F0340921E0385EB93E0EC
:142A5C00F201E80FF91F20802092B3032090840384E6829D9C
:142A7000EC2DFF27E019F10992010AE010E00E94593DE01B80
:142A8400F10B85EB93E0E80FF91F20802092B20380916200D6
:142A9800806880936200DF9A2090B30325BA2090B2032BBAC5
:142AAC0022242092810201C0A895209081022A14D8F322241B
:142AC000209281020027112703D00E94A53D08950E94AB3DF0
:142AD4005801A0925903AA2049F4BB2039F45AD0809162005B
:142AE8008F778093620043C024E630E085010E949A3C0093B1
:142AFC00840385EB93E0E02FFF27E80FF91F20802092B4030F
:142B1000202E8AE0829D10012AE030E085010E949A3C280188
:142B24004218530850921F0340921E0385EB93E0F201E80F24
:142B3800F91F20802092B3032090840384E6829DF501E019BA
:142B4C00F10992010AE010E00E94593DE01BF10B85EB93E0FC
:142B6000E80FF91F20802092B203809162008068809362007B
:142B740003D00E94993D0895DF9A2090AF03222039F020906F
:142B8800B30325BA2090B2032BBA01C001D00895DF9A8FE73C
:142B9C0085BB8FEF8BBB08952090AF03222049F08091620034
:142BB00080688093620022242BBA25BA01C0ECDF08950E94DF
:142BC400AB3D2197A89581E08093AF03AA2439C085EB93E050
:142BD800EA2DFF27E80FF91F20802092B3032092B4032AE022
:142BEC0030E00A2D11270F5F1F4F0E94963CF80185EB93E02A
:142C0000E80FF91F20802092B2032AE030E00A2D11270F5FB3
:142C14001F4F0E94963C18018AE08A9D8001020D131D54DF2D
:142C280008EA11E620E030E00E94323CB1DF00E117E220E025
:142C3C0030E00E94323CA895A3948A2D8A3008F4C3CF2BE4E2
:142C500030E000270E94B0030023B1F000E21EE420E030E02C
:142C64000E94323CA8959CDF00E711E121E030E00E94323C9A
:142C78008FDF00E117E220E030E00E94323CA8951A987894E5
:142C8C000E94B402222420927E023324309229032092280342
:142CA0008091620081608093620001C0A89580917E0288340C
:142CB400D8F3222420927E0281B180718093840320908403D5
:142CC80081B18071821521F480917E028230B0F380917E02B2
:142CDC00823098F50E94C302222420927E0219C020908403B6
:142CF00081B18071821599F08091280390912903019690934A
:142D04002903809328032090840381B18071821521F020909F
:142D18007E022220B1F320907E02222019F300912803109166
:142D2C00290301501040CEDEA89500EF19E422E030E00E943D
:142D4000323CA89505C088E2888321E00EE02CDE809162002E
:142D54008E7F809362000E9486021A9A00271127B5DE219662
:142D68000E94993D089580EC8093B50389EF8093B60384EA59
:142D7C008093B70380EB8093B80389E98093B90382E980937E
:142D9000BA0382E88093BB0388EF8093BC0380E88093BD03B3
:142DA40080E98093BE0388E88093BF0383E88093C00386ECE6
:142DB8008093C10381EA8093C20386E88093C3038EE880931D
:142DCC00C4038CE88093C5038FEF8093C6038093C703089509
:142DE0000E94AE3DC22EA02E26978AE090E0998388832C2D7D
:142DF40033278E010E5F1F4F0E94843E0A810E9402022B80C7
:142E0800222019F0022D0E9402020FE20E9402028AE090E025
:142E1C00998388832A2D33278E010E5F1F4F0E94843E0A8171
:142E30000E9402022B80222019F0022D0E9402020FE20E948A
:142E440002028AE090E0998388832A8533272053384F8E01E3
:142E58000E5F1F4F0E94843E0A810E9402020B810E940202C4
:142E6C000C810E9402020D810E94020226960E94A53D08950E
:142E80000E94AE3DA22EC02E26978AE090E0998388832C2DDC
:142E940033278E010E5F1F4F0E94843E2A80222019F400E326
:142EA8000E9402022A80222019F0022D0E9402022B802220B9
:142EBC0019F0022D0E9402020AE30E9402028AE090E099839B
:142ED00088832A2D33278E010E5F1F4F0E94843E2B80222077
:142EE40019F400E30E9402022A80222019F400E30E940202C2
:142EF8002A80222019F0022D0E9402022B80222019F0022DD7
:142F0C000E9402020AE30E9402028AE090E0998388832A85C8
:142F200033278E010E5F1F4F0E94843E2B80222019F400E398
:142F34000E9402022A80222019F400E30E9402022A80222075
:142F480019F0022D0E9402022B80222019F0022D0E940202CC
:142F5C0026960E94A53D08950C9936C081E080937D030BEFFB
:142F700010E031D022242092A70320927B020C9929C020924B
:142F8400820315C007EF11E024D01091820301B10071029524
:142F98000F700E94153E2090A703202A2092A703809182031B
:142FAC008F5F8093820380918203883038F307EF11E00BD050
:142FC0000C9B08C02090A70320927B02022D0AD000E2D9D66B
:142FD400089502C00150104000300107D9F708950F3321F0F1
:142FE8000B3211F00D3231F481E08093D40322242092D3031A
:142FFC002090D4032220B1F12090D303222019F40093D20319
:143010000EC08091D303843050F486EE93E0E091D303FF27AB
:14302400E80FF91F802F805380838091D3038F5F8093D30346
:143038008530D1F422242092EA032092D3032092D40381E0B3
:14304C00809381032090E8038AE0829D10014090E70384E680
:14306000849D402C420C2090E903420C4092CA0308950E94B9
:14307400DB3D0E9483020093EB030E94DA03A8950E94F23DFB
:143088001895279700E47BD605EB79D62224209202012092A8
:14309C0094020E946A0222242092810201C0A895809181026F
:1430B0008F3F20F4209002012220B9F380919402813471F0CC
:1430C40020902C0330902D0340902A0350902B034214530471
:1430D80018F40E947B0283C308E112E00E940602209002013B
:1430EC00222009F4F9C22090E603222009F47FC00091940298
:143100000E9402020AE00E9402020CEF11E00E9406020AE005
:143114000E9402020AE00E9402020FED11E00E9406020AE0F0
:143128000E9402020FEC11E00E9406022090900228822091BA
:14313C008F0200918E024EDE0AE00E94020207EC11E00E948B
:14315000060220909302288220919202009191028FDE80918D
:143164009402863531F488E2888324E00EE01ADC1DC3809193
:143178009402813431F088E2888325E00EE010DC13C324E1A8
:14318C0000918F023EDC01C0A895809181028230D8F324E1DF
:1431A00000918E0234DC01C0A895809181028230D8F324E1D6
:1431B400009190022ADC01C0A895809181028630D8F324E1C6
:1431C8000091910220DC01C0A895809181028230D8F324E1BF
:1431DC000091920216DC01C0A895809181028230D8F324E1B4
:1431F000009193020CDCA895DBC280919402813409F0ADC120
:14320400209092022092F204209093022092F10420908E029E
:143218002092F40420908F022092F504209090022092F6041E
:14322C00822D99278053984F9093AA028093A9022DE430E0B7
:1432400000270E94B003802F8078803809F03FC00E94B40849
:14325400202E2DE430E000272F920E94B0032F904090910298
:14326800420C802F8F77480E242C2092840387E1841508F572
:14327C002090F40428822091F5040091A9021091AA020E9417
:14329000200998012F5F3F4F8E010F5F1F4F0E9472098D81B6
:1432A4009E81805D97408093F6042B803C802092F50429807B
:1432B8003A802092F40418E1009184030E94413D0093F304E3
:1432CC005CC02DE430E000270E94B003802F8F7790919102CC
:1432E000985E981B292E20928403983108F040C02090F40438
:1432F40028822091F5040091A9021091AA020E942009980185
:14330800215030408E010F5F1F4F0E94720918E10091840337
:14331C000E94413D0093F3040E94B4082090F304200E87E158
:14333000821580F429803A8028822B810D811E810E942009CD
:1433440098012F5F3F4F8E010F5F1F4F0E9472098D819E810B
:14335800805D97408093F6042B803C802092F50429803A802B
:14336C002092F4040E94B408202E00918403020D18E10E9435
:14338000413D0093F3042090E403222079F02090F40428829D
:143394002091F5040091F60411270053184F0E940F0501E067
:1433A8000E94750501E40E9402020AE00E9402020CEF11E0EE
:1433BC000E9406020AE00E9402020AE00E9402020FED11E046
:1433D0000E9406020AE00E9402020FEC11E00E940602209069
:1433E4009002288220918F0200918E02F7DC0AE00E940202D3
:1433F80007EC11E00E9406022090930228822091920200916E
:14340C00910238DD0AE00E9402020AE00E9402020CEA11E0FD
:143420000E9406020AE00E9402020FEC11E00E940602209018
:14343400F60428822091F5040091F404CFDC0AE00E94020272
:1434480007EC11E00E9406022090F10428822091F20400915B
:14345C00F30410DD0AE00E9402022090F60428822090F704E9
:1434700085E0829D90012550304020563F4F00270E949703E7
:143484000E94D0032090F50428822090F70485E0829D9001AC
:14349800255030402F553F4F00270E9497030E94D0032090A1
:1434AC00F40428822090F70485E0829D9001255030402E5542
:1434C0003F4F00270E9497030E94D0032090940228822090F2
:1434D400F70485E0829D9001255030402D553F4F00270E9416
:1434E80097030E94D00381E088832090F70485E0829D900195
:1434FC00255030402C553F4F00270E9497030E94D003209040
:14351000A803222009F44CC13FDB00E513EC20E030E00E9400
:14352400323C84E1888326E002E13CDA84E1888320E102E162
:1435380037DA84E1888325E002E132DA88E2888321E002E1B1
:14354C002DDA24DB00E513EC20E030E00E94323C29C1809166
:143560009402863509F060C005E40E94020204E30E940202D1
:143574002090F60428822090F70485E0829D9001255030404A
:1435880020563F4F00270E9497030E94D0032090F504288200
:14359C002090F70485E0829D9001255030402F553F4F00273D
:1435B0000E9497030E94D0032090F40428822090F70485E0F4
:1435C400829D9001255030402E553F4F00270E9497030E9448
:1435D800D0032090940228822090F70485E0829D90012550E7
:1435EC0030402D553F4F00270E9497030E94D00384E0888304
:143600002090F70485E0829D9001255030402C553F4F0027DB
:143614000E9497030E94D00388E2888324E00EE0C1D9C4C06C
:1436280005E40E94020205E30E9402022090F604288220906D
:14363C00F70485E0829D90012550304020563F4F00270E94B8
:1436500097030E94D0032090F50428822090F70485E0829DD5
:143664009001255030402F553F4F00270E9497030E94D003F2
:143678002090F40428822090F70485E0829D90012550304047
:14368C002E553F4F00270E9497030E94D00385EE8883209013
:1436A000F70485E0829D9001255030402D553F4F00270E9448
:1436B40097030E94D00385E088832090F704829D90012550B3
:1436C80030402C553F4F00270E9497030E94D00388E2888322
:1436DC0025E00EE063D966C009EA11E00E9406020AE00E946B
:1436F000020206E811E00E9406020AE00E9402022090F604FF
:1437040028822090F70485E0829D90012550304020563F4F5E
:1437180000270E9497030E94D0032090F50428822090F704C7
:14372C0085E0829D9001255030402F553F4F00270E9497031A
:143740000E94D0032090F40428822090F70485E0829D9001EE
:14375400255030402E553F4F00270E9497030E94D00383EE22
:1437680088832090F70485E0829D9001255030402D553F4F8D
:14377C0000270E9497030E94D00383E088832090F70485E0E3
:14379000829D9001255030402C553F4F00270E9497030E947C
:1437A400D00388E2888323E00EE0FCD8222420923203209225
:1437B80031032092330320922E0320922F032092300300E451
:1437CC00F0D205EBEED20E947B0222242092E6032092AD0216
:1437E00004EF0E940202279608952AE230E000270E94B0034A
:1437F400202E3324442455243092D1022092D0025092D3026B
:143808004092D20288E090E08A93810192010E94093E109370
:14381C001F0300931E032BE230E000270E94B003009384030F
:14383000202E332440901E0350901F03420C531C50921F032B
:1438440040921E03C2018839E8E09E0728F084E59BE08415F7
:14385800950538F480E09AE090931B0380931A0308C02090D3
:14386C001E0330901F0330921B0320921A0320901A03309009
:143880001B03442455243092C1022092C0025092C3024092C3
:14389400C2024090C2025090C3022090C0023090C10284E6C4
:1438A80090E0A0E0B0E05A924A923A922A928C019D010E946F
:1438BC00693D86E090E0A0E0B0E03A932A931A930A938C010B
:1438D0009D010E94693D1801290180E092E0A0E0B0E0280EA3
:1438E400391E4A1E5B1E8AE090E08A93810192010E941B3E91
:1438F8001093C1020093C0023093C3022093C20280EE98EC10
:14390C00A0E1B0E03A932A931A930A938C019D010E94D03CE9
:143920001093D1020093D0023093D3022093D20218013092BE
:143934001903209218034090C2025090C3022090C00230902B
:14394800C10280E19DECAEE0B0E05A924A923A922A928C01C3
:14395C009D010E94D03C1093D1020093D0023093D3022093E5
:14397000D202180130921703209216034090C2025090C30276
:143984002090C0023090C10288EA97E0AFE0B0E05A924A926A
:143998003A922A928C019D010E94D03C1093D1020093D002DF
:1439AC003093D3022093D2021801309215032092140308958F
:1439C0000E94AB3D2197A89521E530E000270E94B0030023BF
:1439D40059F020E530E000270E94B003002321F081E090E000
:1439E8005C0102C0AA24BB24A092E40328E430E000270E9401
:1439FC00B003202E2BE430E000272F920E94B0032F90209EDD
:143A100000926F0323E330E000270E94B0030093D60327E396
:143A240030E000270E94B0030093E3032CE330E000270E94A1
:143A3800B0030093A8032FE330E000270E94B00300935703FE
:143A4C0020E430E000270E94B0030093560321E430E00027AE
:143A60000E94B0030093550327E430E000270E94B0030093E8
:143A740072032FE430E000270E94B0030093E20381E080933E
:143A88003603A0905703BB24AA2011F4BB2051F0C501813026
:143A9C00E0E09E0761F08230E0E09E0779F01BC0222420920D
:143AB000780389E18093770317C084E1809378038AE0809349
:143AC400770310C02CE430E000270E94B003802F865F809361
:143AD800780385E18093770303C0222420927803A0905603AD
:143AEC00BB24AA2011F4BB2051F0C5018130E0E09E0761F0CF
:143B00008230E0E09E0779F01BC022242092760389E1809368
:143B1400770317C084E1809376038AE08093750310C02CE486
:143B280030E000270E94B003802F865F8093760385E1809364
:143B3C00750303C02224209276032090E403222009F000C136
:143B50002AE330E000270E94B003002309F45FC02090D00306
:143B6400222009F05AC020E330E000270E94B0030093AE0325
:143B780022E330E000270E94B0030093CF03202E87E6829D69
:143B8C00800100571E4F24E630E00E949A3C0093CE0320903A
:143BA000CF038EE6829D800106571D4F24E630E00E949A3CD0
:143BB4000093CD0325E330E000270E94B0030093D70326E48F
:143BC80030E000270E94B0030093AD032EE330E000270E9430
:143BDC00B0030093AC032EE230E000270E94B0030093650349
:143BF0002AE430E000270E94B0030093700323E530E00027E2
:143C04000E94B0030093AF0325E530E000270E94B0030093E9
:143C1800B003A89559C02FE230E000270E94B0030093AE03AE
:143C2C0021E330E000270E94B0030093CF03202E87E6829DB5
:143C4000800100571E4F24E630E00E949A3C0093CE03209085
:143C5400CF038EE6829D800106571D4F24E630E00E949A3C1B
:143C68000093CD0324E330E000270E94B0030093D70325E4DC
:143C7C0030E000270E94B0030093AD032DE330E000270E947C
:143C9000B0030093AC032DE230E000270E94B0030093650395
:143CA40029E430E000270E94B0030093700322E530E000272F
:143CB8000E94B0030093AF0324E530E000270E94B003009336
:143CCC00B003A895222430905603231478F42EE430E00027A9
:143CE0000E94B003002341F48091AC03873C20F481E090E0BB
:143CF4005C0102C0AA24BB24A0923C0320905603222021F023
:143D08008091AC03873C11F405EB4DD08091E303813011F069
:143D1C00833081F42090AF03222021F42090B003222041F0DC
:143D30001A9A82B3886482BB81E08093350316C01A9882B304
:143D4400877B82BB2224209235030EC02090F404288220912B
:143D5800F5040091A9021091AA020E940F0501E00E94750522
:143D6C002090AF03222029F4809162008F77809362002196DD
:143D80000E94993D0895043B11F4C59A0FC0053B11F4C49A05
:143D94000BC0003211F4959807C0003411F4969803C00038C3
:143DA80009F497980895043B11F4C5980FC0053B11F4C4982D
:143DBC000BC0003211F4959A07C0003411F4969A03C0003897
:143DD00009F4979A089528E130E000270E94B003202E3324DA
:143DE400442455243092D1022092D0025092D3024092D20274
:143DF80088E090E08A93810192010E94093E1093C9020093C3
:143E0C00C8023093CB022093CA0288E090E08A930E94093EEB
:143E20001093C9020093C8023093CB022093CA0229E130E09A
:143E340000270E94B003202E3324442455243092D102209231
:143E4800D0025092D3024092D20288E090E08A93810192012D
:143E5C000E94093E1093D1020093D0023093D3022093D2026F
:143E70008090CA029090CB026090C8027090C902600E711EF3
:143E8400821E931E7092C9026092C8029092CB028092CA0283
:143E98002AE130E000270E94B003202E332444245524309237
:143EAC00D1022092D0025092D3024092D2028090CA02909052
:143EC000CB026090C8027090C902620C731C841C951C70924C
:143ED400C9026092C8029092CB028092CA0208952BE130E0CD
:143EE80000270E94B003202E3324442455243092D10220927D
:143EFC00D0025092D3024092D20288E090E08A938101920179
:143F10000E94093E1093C5020093C4023093C7022093C602EA
:143F240088E090E08A930E94093E1093C5020093C402309325
:143F3800C7022093C6022CE130E000270E94B003202E3324F3
:143F4C00442455243092D1022092D0025092D3024092D2020A
:143F600088E090E08A93810192010E94093E4090C6025090E2
:143F7400C7022090C4023090C502200E311E421E531E309263
:143F8800C5022092C4025092C7024092C6022DE130E000275C
:143F9C000E94B003202E3324442455243092D1022092D0021D
:143FB0005092D3024092D2028090C6029090C7026090C40229
:143FC4007090C502620C731C841C951C7092C5026092C40253
:143FD8009092C7028092C6020895219785B78F7D85BFA895F2
:143FEC0089E88093610088E08093620000EA16E821E030E006
:144000000E94323CA8952CD10E94CC150E946A0200E8B9DE52
:1440140000EA16E821E030E00E94323CA895222420927903DE
:1440280005E00E943B02D3DE59DF1A9A00EA16E821E030E02A
:14403C000E94323CA8952090A803222011F00E94E115B8DC59
:144050002224332430922B0320922A032090E403222071F0B6
:144064002090F40428822091F5040091A9021091AA020E9421
:144078000F0501E00E9475052196089580917C03813039F461
:14408C000E94480200E28DDE222420927C03349B5CC00E94E3
:1440A0004B0220901603309017030215130508F052C022249D
:1440B4002092C803809162008F7780936200332430922B0346
:1440C80020922A0320928403A89580912A0390912B03813051
:1440DC00E0E09E07C0F305E00E94550220901403309015033B
:1440F0000215130580F530D0A8950FC02090840333244090AE
:144104002A0350902B032414350428F4822D8F5F80938403A8
:14411800A89580912A0390912B038A30E0E09E0748F3A89532
:14412C0005E00E94550220901403309015030215130550F48F
:1441400081E08093790380916200877F8093620024D001C0D8
:1441540046DF08951A980E941A3B0E946C3B22242ABA27BA98
:1441680024BA21BA22B888E080936100209264002BBA8FE466
:14417C0088BB25BA22BA23B884E5809362008EE18093650091
:144190000E947B020E944602089585B7886185BF85B78062EE
:1441A40085BF0E944602A89557C08895A8952090AF02222088
:1441B80029F00E946D0722242092AF021AE00091F1040E94F9
:1441CC00413D002309F03FC005E00E945502209018033090DD
:1441E00019032016310698F589E88093610088E080936200F3
:1441F4002224332430922B0320922A03209284030FC0209093
:144208008403332440902A0350902B032414350428F4822D7D
:14421C008F5F80938403A89580912A0390912B038A30E0E0C2
:144230009E0748F305E00E94550220901803309019032016DF
:14424400310610F4CCDE01C085DF0E94460220907903222004
:1442580009F401C0A8CF08958FEF8ABB81EB87BB8FEF84BB52
:14426C008BEE81BB8EE482B92224209264002BBA8CE488BBE8
:1442800025BA84E182BB23B88CE58093620087E08093650009
:14429400959A969A979A0895A89581B5886181BDA8958FE0A3
:1442A80081BD0895A89581B5886181BD222421BCA895089590
:1442BC000E94DB3D0E94FE0122242092B00203D00E94F23D45
:1442D00018950E94AB3D2897A89520908803222011F40C9485
:1442E400C929A22CBB24C5018E3CE0E09E0709F4DAC48EEC1D
:1442F8008A159B050CF432C0C501803BE0E09E0709F44CC092
:14430C00813BE0E09E0709F447C0823BE0E09E0709F442C057
:14432000833BE0E09E0709F40CC1843BE0E09E0709F407C1B3
:14433400853BE0E09E0709F402C1803BE0E09E0714F40C94C8
:144348008235C501883CE0E09E0709F4EEC18B3CE0E09E07E3
:14435C0009F470C30C948235C5018D3EE0E09E0709F408C605
:144370008DEE90E08A159B0544F0C501863EE0E09E0709F4EF
:14438400EFC60C948235C5018D3FE0E09E0709F471C58E3F22
:14439800E0E09E0709F46BC60C94823520902001332420944B
:1443AC00309422FE2CC08FEE93E0E0912803F0912903E80FFD
:1443C000F91F20907B02208220907B0230908003322430927A
:1443D400800380912803909129038F3FE0E09E0739F4809158
:1443E80020018460809320010C9482358091280390912903A8
:1443FC00019690932903809328030C9482352090200133240A
:144410002094309423FE1CC080917B02813F71F4809120013E
:1444240088608093200120907B02309080033224309280035D
:144438000C94823580912001807F8093200103EF0E9402021C
:14444C000C94823520907B0230908003321409F048C08FEED1
:1444600093E0998388832091EE0300270E9472030E94D00359
:144474008091EE038F5F8093EE038091ED0381508093ED036B
:1444880022243324309229032092280380912001807F809374
:14449C002001209280032090ED032220E9F42090E40322201E
:1444B00079F02090F40428822091F5040091F604112700537D
:1444C400184F0E940F0501E00E9475052224209288033324F0
:1444D80030922903209228032092830302EF0E9402020C9496
:1444EC00823503EF0E9402028091EC0381508093EC038823EF
:1445000089F480912001807F809320012224209288033324EB
:144514003092290320922803209283030C9482358091200107
:14452800807F80932001222433243092290320922803209232
:14453C0080030C94823580917B02813F49F430908003382665
:144550003092800381E0809389031FC0809189038130D9F418
:1445640020907B0230908003321469F0222420927F03209208
:144578008003209289032092880303EF0E94020208C081E070
:14458C0080937F032224209280032092890380917F03813089
:1445A00009F03FC02090200133242094309422FE38C0A8951A
:1445B40080918803833B61F480E091E090931D0380931C03FE
:1445C800809120018460809320011FC080918803843B61F406
:1445DC0080E094E090931D0380931C03809120018460809359
:1445F00020010FC080918803853B59F480E099E090931D0302
:1446040080931C038091200184608093200102EF0E9402028F
:144618000E94D00300EF0E94020280917F03813011F00C949F
:14462C0082352090200122FE01C002C00C94823580917B026A
:14464000823F81F48091ED0381508093ED0380911C0390910A
:144654001D0380509F4F90931D0380931C0309C080917B02A8
:14466800833F29F48091EC0381508093EC0322243090ED0396
:14467C00231408F04AC03090EC03231408F045C020901C033F
:1446900030901D0330921F0320921E031AC020911E03309112
:1446A4001F0300270E94B003009384033090800330263092EF
:1446B80080030E940202A89580911E0390911F030196909359
:1446CC001F0380931E0380911C0390911D0380509F4F2090A5
:1446E0001E0330901F0328163906C8F281EF90E02090800379
:1446F4003324282639262092800301EF0E94020200918003CF
:144708000E9402022224209280030C94823580912001807FF4
:14471C0080932001222420927F0320928003209288030C94C9
:14473000823580912803909129030196909329038093280311
:14474400A8958130E0E09E070CF46FC18AE190E02090280328
:1447580030902903821593050CF465C1910102E010E00E9406
:14476C00593DF8018AE890E0E80FF91F05901490F0010994F2
:1447800020907B0220923D0352C120907B0220923E034DC1C5
:1447940020907B0220923F0348C120907B022092400343C1C1
:1447A80020907B02209241033EC120907B022092420339C1BD
:1447BC0020907B022092430334C120907B02209244032FC1B9
:1447D00020907B02209245032AC120907B022092460325C1B5
:1447E40020907B022092470320C120907B02209248031BC1B1
:1447F80020907B022092490316C120907B0220924A0311C1AD
:14480C0020907B0220924B030CC120907B0220924C0307C1A8
:1448200020907B0220924D0302C120907B0220924E03FDC0A5
:1448340020907B0220924F03F8C020907B0220925003F3C0A2
:1448480020907B0220925103EEC020907B0220925203E9C09E
:14485C0020907B0220925303E4C020907B0220925403DFC09A
:1448700020907B0230908003321409F0CDC020903D0328825E
:144884002FE230E000270E9497030E94D00320903E0328828C
:1448980020E330E000270E9497030E94D00320903F03288285
:1448AC0021E330E000270E9497030E94D0032090400328826F
:1448C00022E330E000270E9497030E94D00320904103288259
:1448D40024E330E000270E9497030E94D00320904203288242
:1448E80025E330E000270E9497030E94D0032090430328822C
:1448FC002DE230E000270E9497030E94D00320904403288210
:144910002EE230E000270E9497030E94D003209045032882F9
:1449240025E430E000270E9497030E94D003209046032882EB
:1449380026E430E000270E9497030E94D003209047032882D5
:14494C002DE330E000270E9497030E94D003209048032882BA
:144960002EE330E000270E9497030E94D003A8952090490311
:14497400288221E430E000270E9497030E94D00320904A039B
:14498800288229E430E000270E9497030E94D00320904B037E
:14499C0028822AE430E000270E9497030E94D00320904C0368
:1449B000288222E530E000270E9497030E94D00320904D035A
:1449C400288223E530E000270E9497030E94D00320904E0344
:1449D800288224E530E000270E9497030E94D00320904F032E
:1449EC00288225E530E000270E9497030E94D0030E94E01C7D
:144A00002224332430922903209228032092880302EF0E946A
:144A140002020BC003EF0E94020222243324309229032092EA
:144A280028032092880320907B023090800332243092800307
:144A3C000C948235809128039091290301969093290380938D
:144A500028038130E0E09E070CF41EC182E190E02090280384
:144A640030902903821593050CF414C1910102E010E00E9448
:144A7800593DF8018EEB90E0E80FF91F05901490F0010994DC
:144A8C0020907B0220923D0301C120907B0220923E03FCC059
:144AA00020907B0220923F03F7C020907B0220924003F2C056
:144AB40020907B0220924103EDC020907B0220924203E8C052
:144AC80020907B0220924303E3C020907B0220924403DEC04E
:144ADC0020907B0220924503D9C020907B0220924603D4C04A
:144AF00020907B0220924703CFC020907B0220924803CAC046
:144B040020907B0220924903C5C020907B0220924A03C0C041
:144B180020907B0220924B03BBC020907B0220924C03B6C03D
:144B2C0020907B0230908003321409F0A4C020903F032092BE
:144B4000D603288223E330E000270E9497030E94D003209040
:144B540041032092840328822AE330E000270E9497030E9404
:144B6800D003209042032092570328822FE330E000270E94D0
:144B7C0097030E94D0032090430320925603288220E430E057
:144B900000270E9497030E94D0032090440320927203288271
:144BA40027E430E000270E9497030E94D00320904503209260
:144BB800A80328822CE330E000270E9497030E94D0032090ED
:144BCC00460320928403288228E430E000270E9497030E9488
:144BE000D003209048032092840328822DE430E000270E9426
:144BF40097030E94D0032090490320928403288221E530E0A9
:144C080000270E9497030E94D00320904A03209284032882E0
:144C1C0021E430E000270E9497030E94D00320904B032092E7
:144C3000840328822CE430E000270E9497030E94D0030E94A5
:144C4400E01C2090E403222071F02090F40428822091F5042A
:144C58000091A9021091AA020E940F0501E00E9475052224C6
:144C6C00332430922903209228032092880302EF0E9402023E
:144C80000BC003EF0E94020222243324309229032092280355
:144C94002092880320907B02309080033224309280030C9424
:144CA800823580912803909129030196909329038093280394
:144CBC008130E0E09E070CF4D0C082E190E0209028033090D0
:144CD0002903821593050CF4C6C0910102E010E00E94593D53
:144CE400F80182EE90E0E80FF91F05901490F001099420905D
:144CF8007B0220923D03B3C020907B0220923E03AEC0209088
:144D0C007B0220923F03A9C020907B0220924003A4C0209083
:144D20007B02209241039FC020907B02209242039AC020907F
:144D34007B022092430395C020907B022092440390C020907B
:144D48007B02209245038BC020907B022092460386C0209077
:144D5C007B022092470381C020907B02209248037CC0209073
:144D70007B022092490377C020907B0220924A0372C020906F
:144D84007B0220924B036DC020907B0220924C0368C020906B
:144D98007B0230908003321409F056C0222433243092290367
:144DAC00209228032092880302EF0E94020220903D032092A0
:144DC000840328822BE430E000270E9497030E94D003209007
:144DD4003E0320928403288220E530E000270E9497030E948D
:144DE800D00320903F032092840328822EE430E000270E9424
:144DFC0097030E94D0032090400320928403288222E430E0A8
:144E100000270E9497030E94D00320904103209284032882DF
:144E24002FE430E000270E9497030E94D003209042032092D8
:144E38008403288227E330E000270E9497030E94D0030E94A1
:144E4C00E01C0BC003EF0E94020222243324309229032092B6
:144E600028032092880320907B0230908003322430928003CB
:144E74000C948235A89520907A03222009F43EC00E948635CF
:144E880020907F03222049F122242092840319C020908403D9
:144E9C00209286038BE893E0E22DFF27E80FF91F2080288253
:144EB00020918403332700270E9497030E94D00380918403EC
:144EC4008F5F8093840380918403883118F302EF0E9402025F
:144ED800222420927F030C948235222420927F03209288033E
:144EEC003324309229032092280303EF0E9402020C948235A1
:144F000080912803909129038931E0E09E0791F422243324D3
:144F1400309229032092280320907B02309080033224309236
:144F2800800381E080937A030C948235809128039091290321
:144F3C008931E0E09E0710F00C94823520907B02309080037B
:144F50003224309280038BE893E0E0912803F09129033197BB
:144F6400E80FF91F2082809128039091290301969093290319
:144F7800809328030C948235A8958091280390912903019633
:144F8C0090932903809328038130E0E09E0791F08230E0E07B
:144FA0009E0791F08330E0E09E07B1F08430E0E09E0709F408
:144FB40057C08530E0E09E0791F052C020907B022092B7028D
:144FC80020907B022092B80222242092F10446C020907B021C
:144FDC002092B60241C020907B0230908003321481F520907A
:144FF000B7022092F3042090B8022092F2042090B602288227
:145004002FE130E000270E9497030E94D00322243324309241
:145018002903209228032092880302EF0E9402022090E40310
:14502C002220D1F02090F40428822091F5040091A902109194
:14504000AA020E940F0501E00E9475050BC003EF0E9402029A
:145054002224332430922903209228032092880320907B0276
:14506800309080033224309280030C948235A8958091280386
:14507C0090912903019690932903809328038130E0E09E0799
:1450900091F08230E0E09E0799F08330E0E09E07A1F084308E
:1450A400E0E09E0709F453C08530E0E09E0781F04EC020903A
:1450B8007B022092B90249C020907B022092BA0244C02090A2
:1450CC007B022092BB023FC020907B0230908003321471F5C9
:1450E0002090B9022092F6042090BA022092F5042090BB0221
:1450F4002092F4040E945A080093F7048091F60499278053CE
:14510800984F9093AA028093A90222243324309229032092E2
:14511C002803209288032FE130E000270E94B003013011F445
:145130000E94B40802EF0E9402020BC003EF0E9402022224CD
:14514400332430922903209228032092880320907B0230900B
:1451580080033224309280030C948235809128039091290345
:14516C00019690932903809328038130E0E09E0771F08230E2
:14518000E0E09E0779F08330E0E09E0709F4F8C08430E0E00C
:145194009E0759F0F3C020907B0220928403EEC020907B0225
:1451A80020928603E9C020907B0230908003321409F0D7C0C9
:1451BC002090840328822AE230E000270E9497030E94D0030A
:1451D0002090860328822BE230E000270E9497030E94D003F3
:1451E400209084033324322C222430921B0320921A03209026
:1451F8008603332440901A0350901B03420C531C50921B031B
:14520C0040921A03222430922903209228032092880302EF60
:145220000E94020220901A0330901B03442455243092C102C3
:145234002092C0025092C3024092C2024090C2025090C3027C
:145248002090C0023090C10284E690E0A0E0B0E05A924A92AB
:14525C003A922A928C019D010E94693D86E090E0A0E0B0E05D
:145270003A932A931A930A938C019D010E94693D18012901A0
:1452840080E092E0A0E0B0E0280E391E4A1E5B1E8AE090E0EC
:145298008A93810192010E941B3E1093C1020093C002309357
:1452AC00C3022093C20280EE98ECA0E1B0E03A932A931A9378
:1452C0000A938C019D010E94D03C1093D1020093D0023093C6
:1452D400D3022093D202180130921903209218034090C20212
:1452E8005090C3022090C0023090C10280E19DECAEE0B0E010
:1452FC005A924A923A922A928C019D010E94D03C1093D102FF
:145310000093D0023093D3022093D20218013092170320925E
:1453240016034090C2025090C3022090C0023090C10288EABC
:1453380097E0AFE0B0E05A924A923A922A928C019D010E94AE
:14534C00D03C1093D1020093D0023093D3022093D20218012E
:1453600030921503209214030BC003EF0E9402022224332496
:1453740030922903209228032092880320907B0230908003AD
:145388003224309280030C94823580917B02813F69F43090B4
:14539C00800338263092800381E080938903222420928A0352
:1453B0000C94823520908303222011F40C94D73380917B02DD
:1453C400823F51F4222433243092290320922803209283032F
:1453D8000C9482350E94863520907F03222011F40C94C933F8
:1453EC00222420927F03A0908303BB24C501843CE0E09E07B3
:1454000009F4E5C2853CE0E09E0709F4EAC2863CE0E09E07FE
:1454140009F488C3873CE0E09E0709F48FC38A3CE0E09E079A
:1454280009F48CC48C3CE0E09E0709F449C58F3CE0E09E07BB
:14543C0009F45AC68FEC8A159B0544F1C501803AE0E09E076B
:1454500009F45AC0813AE0E09E0709F4EDC0823AE0E09E0746
:1454640009F400C1843AE0E09E0709F413C1803AE0E09E0763
:1454780014F40C948235C501883BE0E09E0709F473C1893BDE
:14548C00E0E09E0709F4CFC10C948235C501853EE0E09E07D5
:1454A00009F46CC7873EE0E09E0709F49DC7893EE0E09E0711
:1454B40009F4E4C78A3EE0E09E0711F40C94AD328AEE90E0A3
:1454C8008A159B0544F0C501853DE0E09E0709F42DC70C94DF
:1454DC008235C5018A3FE0E09E0711F40C94B8328B3FE0E0F8
:1454F0009E0711F40C94C0328C3FE0E09E0711F40C94BF33A5
:145504000C9482350091F504005D0E9402020FE20E94020218
:145518000091F404005D0E9402020FE20E9402020091F604D1
:14552C00005D0E94020200E20E94020200E20E9402021AE05E
:145540000091F3040E94433D00938403005D0E9402022090E0
:1455540084038AE0829D2090F30433242018310830921F03E0
:1455680020921E03022D005D1F4F0E9402020AE30E94020229
:14557C001AE00091F2040E94433D00938403005D0E9402025B
:14559000209084038AE0829D2090F204332420183108309217
:1455A4001F0320921E03022D005D1F4F0E9402020AE30E94CF
:1455B80002021AE00091F1040E94433D00938403005D0E9420
:1455CC000202209084038AE0829D2090F1043324201831089A
:1455E00030921F0320921E03022D005D1F4F0E9402020AE076
:1455F4000E9402020091F5040E9402020091F4040E9402029E
:145608000091F6040E9402020091F3040E9402020091F204A8
:14561C000E9402020091F1040E94020202EF0E9402022224CB
:14563000209283030C94823502EF0E94020281E08093E603E3
:145644002224332430922B0320922A038093AD0289E790E044
:1456580090932D0380932C03209283030C94823502EF0E9487
:14566C00020222242092E603332430922B0320922A0381E0BE
:145680008093AD0280E19EE090932D0380932C0320928303A8
:145694000C94823502EF0E940202A8952AE230E000270E94F2
:1456A800B003009366032BE230E000270E94B00300935E03B2
:1456BC002224332430921D0320921C0313C08FEE93E0E09156
:1456D0001C03F0911D03E80FF91F8FEF808380911C03909125
:1456E4001D03019690931D0380931C0380911C0390911D0315
:1456F8008030E1E09E0728F322242092840315C0A8958FEE5F
:14570C0093E0998388832091840300270E9472030E94D00304
:145720000E94D0030E94D003809184038F5F8093840380915A
:1457340084038D3038F32090660328822AE230E000270E944A
:1457480097030E94D00320905E0328822BE230E000270E949D
:14575C0097030E94D0030C9400002224209283030C948235B5
:1457700002EF0E940202A89500EF0E9402028091F7048A5FC7
:145784008093840337C017E0009184030E94413D0093660355
:1457980022242092690323C02090660385E0829D9001205612
:1457AC003F4F209069033324220D331D00270E94B003202E9F
:1457C000332430921F0320921E03409080035524422453241E
:1457D400409280030E940202809169038F5F809369038091CB
:1457E80069038530C8F2809184038150809384038091F704C3
:1457FC00815020908403821508F4C1CF81EF90E0209080035B
:145810003324282639262092800301EF0E94020200918003A1
:145824000E9402022224209283030C94823502EF0E9402025E
:14583800A89520E630E000270E94B003202E332430921D0306
:14584C0020921C0303E611E00E9406020AE00E940202809152
:145860001C0390911D030996809384039CC01AE0009184032D
:145874000E94413D0093660322242092690329C0209066039E
:1458880086E0829D90012F593F4F209069033324220D331DEE
:14589C0000270E94B003202E332430921F0320921E03409050
:1458B000800355244224532440928003CE010296E091690372
:1458C400FF27E80FF91F2082809169038F5F809369038091FE
:1458D8006903863098F280911E0390911F03807690708030F5
:1458EC00890709F055C02C8028822B810A810E94F01600E6EF
:1459000011E00E940602222428822E810D810E94401700E6EC
:1459140011E00E94060280911E0390911F038F7190705C0112
:145928008130E0E09E07B1F08230E0E09E07B9F08430E0E080
:14593C009E07C1F08830E0E09E07C9F08130E0E09E07FCF029
:14595000C5018031E0E09E07A9F019C005E511E00E94060270
:1459640018C00AE411E00E94060213C00EE311E00E9406026F
:145978000EC003E311E00E94060209C00CE211E00E9406027A
:14598C0004C008E211E00E9406020AE00E9402028091840396
:1459A00081508093840320901C0330901D0340908403552409
:1459B4002414350408F459CFA89504EF0E940202222420927C
:1459C80083030C94823502EF0E9402020E94E11522242092C7
:1459DC0083030C94823502EF0E94020205E00E94550218014C
:1459F000442437FC4094552447FC50943092D1022092D0027B
:145A04005092D3024092D20220901A0330901B0344245524A5
:145A18003092CD022092CC025092CF024092CE024090CE0274
:145A2C005090CF022090CC023090CD028090D2029090D302CF
:145A40006090D0027090D1025A924A923A922A928301940154
:145A54000E94693D1093D1020093D0023093D3022093D202FC
:145A680085E593E0A0E0B0E018012901280E391E4A1E5B1E8C
:145A7C003092D1022092D0025092D3024092D2028BEA96E0B5
:145A9000A0E0B0E0BA93AA939A938A93810192010E94D03C5B
:145AA4001093D1020093D0023093D3022093D20288E090E01C
:145AB8008A930E941B3E0093840300EF0E94020220908403DC
:145ACC0030908003322430928003022D0E9402024090D2026F
:145AE0005090D3022090D0023090D10220928403309080036C
:145AF400322430928003022D0E94020281EF90E0209080031B
:145B08003324282639262092800301EF0E94020200918003A6
:145B1C000E940202222420928303EEC702EF0E940202F89479
:145B30000E94562181E085BF82E085BF0C94003E02EF0E948C
:145B4400020200EF0E940202A89581E090E090931F0380934E
:145B58001E03E3C080911E0390911F038130E0E09E070CF4EA
:145B6C00C7C089E190E020901E0330901F03821593050CF4E2
:145B8000BDC0910102E010E00E94593DF80186E091E0E80F31
:145B9400F91F05901490F00109942FE230E000270E94B00381
:145BA80000938403A7C020E330E000270E94B00300938403BF
:145BBC009FC021E330E000270E94B0030093840397C022E370
:145BD00030E000270E94B003009384038FC024E330E000278E
:145BE4000E94B0030093840387C025E330E000270E94B00363
:145BF800009384037FC02DE230E000270E94B003009384038B
:145C0C0077C02EE230E000270E94B003009384036FC025E45F
:145C200030E000270E94B0030093840367C026E430E0002762
:145C34000E94B003009384035FC02DE330E000270E94B00332
:145C48000093840357C02EE330E000270E94B0030093840360
:145C5C004FC021E430E000270E94B0030093840347C029E466
:145C700030E000270E94B003009384033FC02AE430E0002736
:145C84000E94B0030093840337C022E530E000270E94B00313
:145C9800009384032FC023E530E000270E94B0030093840341
:145CAC0027C024E530E000270E94B003009384031FC025E565
:145CC00030E000270E94B0030093840317C0222420928403D4
:145CD40013C02224209284030FC02224209284030BC022240B
:145CE8002092840307C022242092840303C081EF809384035C
:145CFC002090840330908003322430928003022D0E940202AA
:145D100080911E0390911F03019690931F0380931E038091E9
:145D24001E0390911F038A31E0E09E0708F414CF00918003F4
:145D38000E940202222420928303E0C602EF0E94020200EF07
:145D4C000E940202A89581E090E090931F0380931E03A3C0B3
:145D600080911E0390911F038130E0E09E070CF487C081E1FB
:145D740090E020901E0330901F03821593050CF47DC09101FA
:145D880002E010E00E94593DF80188E391E0E80FF91F059084
:145D9C001490F00109942224209284036BC027E330E00027D6
:145DB0000E94B0030093840363C023E330E000270E94B003BB
:145DC400009384035BC029E330E000270E94B00300938403E4
:145DD80053C02AE330E000270E94B003009384034BC0209036
:145DEC0057032092840346C0209056032092840341C0209017
:145E00007203209284033CC02090A8032092840337C028E44D
:145E140030E000270E94B003009384032FC02BE430E000279F
:145E28000E94B0030093840327C02DE430E000270E94B00373
:145E3C00009384031FC021E530E000270E94B00300938403AD
:145E500017C021E430E000270E94B003009384030FC02CE4DD
:145E640030E000270E94B0030093840307C02224209284033E
:145E780003C081EF80938403209084033090800332243092B7
:145E8C008003022D0E94020280911E0390911F03019690937B
:145EA0001F0380931E0380911E0390911F038231E0E09E070B
:145EB40008F454CF009180030E9402022224209283031EC69F
:145EC8000E941A3B0E946C3B05E00E9455021801442437FCF4
:145EDC004094552447FC50943092D1022092D0025092D3026E
:145EF0004092D20220901A0330901B03442455243092CD02DB
:145F04002092CC025092CF024092CE024090CE025090CF0263
:145F18002090CC023090CD028090D2029090D3026090D002CD
:145F2C007090D1025A924A923A922A92830194010E94693DDD
:145F40001093D1020093D0023093D3022093D20285E593E076
:145F5400A0E0B0E018012901280E391E4A1E5B1E3092D102E3
:145F68002092D0025092D3024092D2028BEA96E0A0E0B0E049
:145F7C00BA93AA939A938A93810192010E94D03C1093D10204
:145F90000093D0023093D3022093D20202EF0E9402020E9440
:145FA400D00300EF0E94020222242092840314C020918403F6
:145FB800332700270E94B003009366033090800330263092A8
:145FCC0080030E940202809184038F5F8093840380918403E0
:145FE000883540F388E090E04090D2025090D3022090D0020A
:145FF4003090D1028A93810192010E941B3E009384033090FF
:1460080080033026309280030E9402024090D2025090D30267
:14601C002090D0023090D102209284033090800332243092C7
:146030008003022D0E9402020091F6040E9402022090F60429
:14604400309080033224309280030091F5040E94020220908A
:14605800F504309080033224309280030091F4040E9402022E
:14606C002090F404309080033224309280030091F3040E9470
:1460800002022090F304309080033224309280030091F204FC
:146094000E9402022090F2043090800332243092800383E06B
:1460A80080938403382630928003082F0E94020283E2809352
:1460BC00840330908003382630928003082F0E94020201EF96
:1460D0000E94020281EF90E02090800333242826392620924D
:1460E4008003022D0E94020222242092830308C502EF0E9472
:1460F800020200EF0E94020281E090E090931F0380931E03B1
:14610C0002C180911E0390911F038130E0E09E070CF4E6C08B
:146120008BE190E020901E0330901F03821593050CF4DCC011
:14613400910102E010E00E94593DF8018AE591E0E80FF91FD3
:1461480005901490F00109942090AF0320928403C9C02090A8
:14615C00B00320928403C4C02090AE0320928403BFC0809195
:14617000CF03873C20F481E090E05C0102C0AA24BB24A092A3
:146184008403B2C02090CF0320928403ADC02090650320921C
:146198008403A8C02090D70320928403A3C02090AD032092CC
:1461AC0084039EC02090AC032092840399C020906F03209235
:1461C000840394C020907003209284038FC02090F4042092EB
:1461D40084038AC02090F5042092840385C02090F604209263
:1461E800840380C02090F304209284037BC02090F204209269
:1461FC00840376C02090F1042092840371C04090C60250904B
:14621000C7022090C4023090C5022092840366C088E090E07D
:146224004090C6025090C7022090C4023090C5028A93810189
:1462380092010E941B3E1093D1020093D0023093D30220939E
:14624C00D20218012901209284034AC088E090E04090D20268
:146260005090D3022090D0023090D1028A93810192010E948C
:146274001B3E0093840338C083E08093840334C083E2809342
:14628800840330C02090E403222021F082E08093840328C0BD
:14629C002AE330E000270E94B0030093840320C02AE330E03E
:1462B00000270E94B003002341F02090D003222021F481E0CF
:1462C40090E05C0102C0AA24BB24A09284030CC02090C8038A
:1462D8002092840307C022242092840303C081EF8093840366
:1462EC002090840330908003322430928003022D0E940202B4
:1463000080911E0390911F03019690931F0380931E038091F3
:146314001E0390911F038C31E0E09E0708F4F5CE009180031C
:146328000E940202222420928303E8C302EF0E94020200EF0C
:14633C000E9402022090B00330908003322430928003022D37
:146350000E94020281EF90E0209080033324282639262092CA
:14636400800301EF0E940202009180030E940202222420925A
:146378008303C4C302EF0E94020200EF0E9402022AE230E0BC
:14638C0000270E94B003009384033090800330263092800389
:1463A0000E9402022BE230E000270E94B003009384033090D0
:1463B40080033026309280030E94020281EF90E020908003FE
:1463C8003324282639262092800301EF0E94020200918003DE
:1463DC000E9402022224209283038EC302EF0E94020200EFB2
:1463F0000E94020283E0809384033090800338263092800310
:14640400082F0E94020283E280938403309080033826309245
:146418008003082F0E94020228E230E000270E94B0030093E7
:14642C008403309080033026309280030E94020229E230E036
:1464400000270E94B0030093840330908003302630928003D4
:146454000E94020281EF90E0209080033324282639262092C5
:14646800800301EF0E940202009180030E9402022224209255
:14647C00830342C302EF0E940202222420928403288228E1B8
:1464900030E000270E9497030E94D0038CE080938403282EB4
:1464A400288229E130E000270E9497030E94D00380E09CE06C
:1464B80080938403282E28822AE130E000270E9497030E9416
:1464CC00D00380E09CE0A0E0B0E09093C9028093C802B093EF
:1464E000CB02A093CA022224209284038FEF80932101809397
:1464F400220180932301809324018093250180E090E0A0E079
:14650800B0E09093C5028093C402B093C702A093C60228827B
:14651C002BE130E000270E9497030E94D00320908403288296
:146530002CE130E000270E9497030E94D00320908403288281
:146544002DE130E000270E9497030E94D003222420928303CF
:14655800D5C202EF0E940202F89461E081E085BF82E085BFE9
:14656C000C94003E02EF0E940202E7D2222420928303C2C2EB
:1465800002EF0E94020200EF0E9402020091F6040E940202AA
:146594002090F604309080033224309280030091F5040E943F
:1465A80002022090F504309080033224309280030091F404CB
:1465BC000E9402022090F4043090800332243092800300910E
:1465D000F3040E9402022090F3043090800332243092800395
:1465E4000091F2040E9402022090F204309080033224309275
:1465F80080032FE130E000270E94B003009384030E940202B0
:14660C00209084033090800332243092800388E090E04090BD
:14662000C6025090C7022090C4023090C5028A9381019201C6
:146634000E941B3E1093D1020093D0023093D3022093D2025D
:14664800180130921D0320921C0388E090E08A930E941B3E82
:14665C00009384030E940202209084033090800332243092D8
:14667000800320901C0330901D0320928403022D0E940202D6
:1466840020908403309080033224309280034090C602509075
:14669800C7022090C4023090C50220928403022D0E9402021A
:1466AC00209084033090800332243092800388E090E040901D
:1466C000CA025090CB022090C8023090C9028A938101920116
:1466D4000E941B3E1093D1020093D0023093D3022093D202BD
:1466E80088E090E08A930E941B3E10931D0300931C03180120
:1466FC0020928403309080033026309280030E9402024090FD
:14671000D2025090D3022090D0023090D102209284033090DE
:146724008003322430928003022D0E9402024090CA025090F2
:14673800CB022090C8023090C90220928403309080033224A9
:14674C0030928003022D0E94020281EF90E0209080033324B5
:14676000282639262092800301EF0E940202009180030E94F7
:146774000202222420928303C3C102EF0E94020281E0809300
:146788008703222420928303B9C103EF0E94020222242092EB
:14679C007F033324309229032092280320928303ABC1809190
:1467B0007B02803F59F481E080938A0322242092800320921E
:1467C4008803209283039CC180918A03813009F090C1209058
:1467D8007B0220928003222420928A03A0907B02BB24C50124
:1467EC00803BE0E09E0794F085ED8A159B0524F102E010E05D
:1468000095010E94593DF80182E390E0E80FF91F05901490A0
:14681400F0010994C501803AE0E09E0709F41DC1813AE0E0A7
:146828009E0709F41CC1823AE0E09E0709F41BC1843AE0E065
:14683C009E0709F41AC160C1C501853EE0E09E0709F44FC1AF
:14685000863EE0E09E0709F4F0C0873EE0E09E0709F441C135
:14686400893EE0E09E0709F430C18A3EE0E09E0709F433C1E8
:146878008D3EE0E09E0709F4C8C0853EE0E09E070CF43CC132
:14688C00C5018A3FE0E09E0709F413C18B3FE0E09E0709F407
:1468A00012C18C3FE0E09E0709F405C18D3FE0E09E0709F4F0
:1468B400A4C08E3FE0E09E0709F4B3C021C180EB80938803DF
:1468C80080912001807F8093200181E08093EE0383E080937C
:1468DC00ED038093EC032224332430922903209228030AC183
:1468F00081EB8093880380912001807F8093200184E08093AE
:14690400EE0385E08093ED0383E08093EC0322243324309262
:14691800290320922803F2C082EB8093880380912001807F74
:14692C008093200189E08093EE0383E08093ED038093EC034E
:14694000222433243092290320922803DBC083EB8093880334
:1469540020907B022092800383E08093ED038093EC0322241F
:1469680033243092290320922803C8C084EB809388032090B4
:14697C007B022092800385E08093ED0383E08093EC03222442
:1469900033243092290320922803B4C085EB8093880320909F
:1469A4007B022092800383E08093ED038093EC032224332428
:1469B8003092290320922803A1C08BEC8093880322243324ED
:1469CC00309229032092280397C08EEC8093880322243324E0
:1469E00030922903209228038DC088EC8093880322243324DC
:1469F400309229032092280383C08DEF8093880381E090E096
:146A0800909329038093280379C08DEE8093880322243324FE
:146A1C0030922903209228036FC08EEF8093880322243324B4
:146A3000309229032092280365C086EE8093880322243324B3
:146A440030922903209228035BC088EB8093830357C089EBC1
:146A58008093830353C080EA809383034FC081EA8093830368
:146A6C004BC082EA8093830347C084EA8093830343C08FEC7A
:146A8000809383033FC08CEC809383033BC085ED8093830353
:146A940037C08AEC8093830333C087EC809383032FC084EC8A
:146AA800809383032BC085EC8093830327C08CEF8093830351
:146ABC0023C08AEF809383031FC08BEF809383031BC089EE8D
:146AD0008093830317C086EC8093830313C08AEE8093830353
:146AE4000FC087EE809383030BC085EE8093830307C0809112
:146AF8007B028F3E19F402EF0E94020228960E94993D0895C9
:146B0C00222420927A032092880333243092290320922803A1
:146B200020907B0230908003321439F481E080937F03222442
:146B34002092800305C0222420927F0320928003089500EF18
:146B48000E94020222243324309229032092280319C02091A1
:146B5C0028033091290300270E94B003009384033090800334
:146B70003026309280030E94020280912803909129030196B0
:146B8400909329038093280380912803909129038831E0E06E
:146B98009E07F8F222243324309229032092280381EF90E012
:146BAC00209080033324282639262092800301EF0E940202D3
:146BC000009180030E94020208950E94B23D269700240B826B
:146BD40011241D820C821A8209820882222420928603209267
:146BE800A30320927F03A89580E09CE0A0E0B0E09093C102B0
:146BFC008093C002B093C302A093C2029AC3209086032220D9
:146C100009F0F4C100EF0E9402022224209280033324309299
:146C240029032092280332C0209128033091290300270E94CF
:146C3800B0030093840330908003302630928003002319F071
:146C4C000E94020216C085E190E02090280330902903821584
:146C6000930550F400E20E94020280E2209080032826209227
:146C7400800303C00B8003940B8280912803909129030196F7
:146C8800909329038093280380912803909129038831E0E069
:146C9C009E0730F2A090F504BB24C5018130E0E09E0709F43C
:146CB00038C08230E0E09E0709F43AC08330E0E09E0709F4B5
:146CC4003CC08430E0E09E0709F43EC08530E0E09E0709F495
:146CD80040C08630E0E09E0709F442C08730E0E09E0709F475
:146CEC0044C08830E0E09E0709F446C08930E0E09E0709F455
:146D000048C08A30E0E09E0709F44AC08B30E0E09E0709F434
:146D14004CC08C30E0E09E0709F44EC053C08AE4E82E81E635
:146D2800A82E8EE6C82E4CC086E4E82E85E6A82E82E6C82EEC
:146D3C0045C08DE4E82E81E6A82E82E7C82E3EC081E4E82EA2
:146D500080E7A82E82E7C82E37C08DE4E82E81E6A82E89E768
:146D6400C82E30C08AE4E82E85E7A82E8EE6C82E29C08AE4AE
:146D7800E82E8CE6A82E89E7C82E22C081E4E82E85E7A82EA4
:146D8C0087E6C82E1BC083E5E82E85E6A82E80E7C82E14C0C5
:146DA0008FE4E82E83E6A82E84E7C82E0DC08EE4E82E8FE6EC
:146DB400A82E86E7C82E06C084E4E82E85E6A82E83E6C82EAE
:146DC80081E090E090931D0380931C0309C080911C03909157
:146DDC001D03019690931D0380931C0380911C0390911D0306
:146DF000883EE3E09E0778F30E2D0E940202209080032E2490
:146E0400209280030A2D0E940202209080032A2420928003B2
:146E18000C2D0E940202209080032C24209280030DE20E943E
:146E2C00020280E2209080032826209280031AE00091F404B3
:146E40000E94433D802F805D80938403082F0E940202209069
:146E54008403309080033224309280031AE00091F4040E94A0
:146E6800433D8AE0809F8091F4048019805D80938403082FBD
:146E7C000E94020220908403309080033224309280030DE258
:146E90000E94020280E22090800328262092800314E60091A5
:146EA400F6040E94433D84E6809F0091F60400191AE00E94F5
:146EB800433D802F805D80938403082F0E940202209084030C
:146ECC00309080033224309280031AE00091F6040E94433D2D
:146EE0008AE0809F8091F6048019805D80938403082F0E9421
:146EF4000202209084033090800332243092800300E20E94ED
:146F0800020280E2209080032826209280031AE00091F304D7
:146F1C000E94433D802F805D80938403082F0E94020220908C
:146F30008403309080033224309280031AE00091F3040E94C4
:146F4400433D8AE0809F8091F3048019805D80938403082FE1
:146F58000E94020220908403309080033224309280030BE37C
:146F6C000E9402028BE3209080032826209280031AE00091BC
:146F8000F2040E94433D802F805D80938403082F0E940202E2
:146F940020908403309080033224309280031AE00091F20453
:146FA8000E94433D8AE0809F8091F2048019805D8093840313
:146FBC00082F0E9402022090840330908003322430928003CF
:146FD00000270E94020222242092840308C000270E940202CC
:146FE400809184038F5F80938403209084030B80201498F3F8
:146FF800A8953CC180918603813009F037C12090A303222077
:14700C00E1F080E092E0A0E0B0E04090C2025090C3022090D4
:14702000C0023090C102281A390A4A0A5B0A3092C1022092A2
:14703400C0025092C3024092C20222242092A30303C02224A2
:14704800209285034090C2025090C3022090C0023090C102CC
:14705C008090CA029090CB026090C8027090C90262187308DD
:147070008408950880E092E0A0E0B0E0681679068A069B06D3
:14708400F8F48090CA029090CB026090C8027090C902621844
:1470980073088408950881E090E0A0E0B0E0680E791E8A1EAA
:1470AC009B1E7092D1026092D0029092D3028092D20213018D
:1470C0003D822C8281E090E09A83898300EF0E94020222247A
:1470D4002092800380E09CE0A0E0B0E04090C2025090C3024E
:1470E8002090C0023090C102281639064A065B0609F0B4C004
:1470FC0021E530E000270E94B003013041F429E131E0002746
:147110000E94B0030093840307C02FE230E000270E94B00398
:1471240000938403009184030E940202A8952090840330904B
:14713800800332243092800380E09CE0A0E0B0E09093C10253
:14714C008093C002B093C302A093C20282E090E09A83898360
:1471600081C088E090E04090C2025090C3022090C002309097
:14717400C1028A93810192010E941B3E1093D1020093D0023C
:147188003093D3022093D20288E090E08A930E941B3E009351
:14719C007E032091C0023091C1020E94B0030093A5030C804B
:1471B0001D8009811A810016110629F50EEE0E9402028EEEA0
:1471C40090E0209080033324282639262092800381E090E00A
:1471D800A0E0B0E04090C2025090C3022090C0023090C10265
:1471EC00280E391E4A1E5B1E3092C1022092C0025092C30281
:147200004092C20237C08091A5038E3E19F422242092A503BB
:147214000091A5030E9402022090A5033090800332243092D4
:14722800800381E090E0A0E0B0E04090C2025090C302209005
:14723C00C0023090C102280E391E4A1E5B1E3092C102209254
:14725000C0025092C3024092C20289819A8101969A83898346
:1472640080E092E009801A80801591050CF077CF81EF90E0D4
:14727800209080033324282639262092800301EF0E94020200
:14728C00009180030E940202A895222420927B0281E090E0B1
:1472A00090931D0380931C0341C081E08093840305C0809193
:1472B40084038F5F80938403809184038436B8F3A89588E114
:1472C8009CE920901C0330901D038215930520F40024039480
:1472DC0008822FC080917B02823F21F481E08093860327C0DD
:1472F00080917B02833F89F4809185038F5F8093850381E03A
:147304008093A30382E0209085038215B0F4002403940882A2
:1473180012C080911C0390911D03019690931D0380931C0312
:14732C0080911C0390911D038034ECE99E0708F4B6CF40905D
:14734000CA025090CB022090C8023090C9028090C2029090C7
:14735400C3026090C0027090C102261437044804590420F0BD
:147368000880002009F44DCC26960E94A83D08950E94AB3DE9
:14737C00A02E2197222420927D0320902601222009F01FC10D
:14739000AA2009F41CC18091B003813009F017C12090250129
:1473A4003090F604321401F185EF80938403282E2882209124
:1473B800C8023091C90200917E030E9497030E94D00305D1D2
:1473CC002090F6042092250128822091C8023091C9020091E9
:1473E0007E030E9497030E94D003F5D0209024013090F50414
:1473F400321401F186EF80938403282E28822091C802309102
:14740800C90200917E030E9497030E94D003DFD02090F5048A
:14741C002092240128822091C8023091C90200917E030E9420
:1474300097030E94D003CFD0209023013090F404321401F1D6
:1474440087EF80938403282E28822091C8023091C90200918C
:147458007E030E9497030E94D003B9D02090F40420922301E7
:14746C0028822091C8023091C90200917E030E9497030E946B
:14748000D003A9D0209022013090F304321401F188EF809360
:147494008403282E28822091C8023091C90200917E030E94A2
:1474A80097030E94D00393D02090F304209222012882209187
:1474BC00C8023091C90200917E030E9497030E94D00383D050
:1474D000209021013090F204321401F189EF80938403282E80
:1474E40028822091C8023091C90200917E030E9497030E94F3
:1474F800D0036DD02090F2042092210128822091C802309110
:14750C00C90200917E030E9497030E94D0035DD08A2D8F3F2B
:1475200021F1A8822091C8023091C90200917E030E949703C6
:147534000E94D0034ED081E090E0A0E0B0E04090C602509057
:14754800C7022090C4023090C502280E391E4A1E5B1E309239
:14755C00C5022092C4025092C7024092C60284EF9FEFA3E013
:14757000B0E04090CA025090CB022090C8023090C9022816EB
:1475840039064A065B0618F081E08093260100E40E94C31EF9
:147598002224332430921D0320921C0309C080911C03909175
:1475AC001D03019690931D0380931C0380911C0390911D032E
:1475C0008032EEE49E0778F300E40E94D71E21960E94993D79
:1475D400089581E090E0A0E0B0E04090CA025090CB0220902C
:1475E800C8023090C902280E391E4A1E5B1E3092C90220928D
:1475FC00C8025092CB024092CA0288E090E08A93810192015A
:147610000E941B3E1093D1020093D0023093D3022093D20271
:1476240088E090E08A930E941B3E00937E0308952197409029
:14763800C6025090C7022090C4023090C502209284032882ED
:14764C002DE130E000270E9497030E94D00388E090E040908C
:14766000C6025090C7022090C4023090C5028A938101920176
:147674000E941B3E1093D1020093D0023093D3022093D2020D
:14768800180129012092840328822CE130E000270E94970348
:14769C000E94D00388E090E04090D2025090D3022090D002B2
:1476B0003090D1028A93810192010E941B3E00938403202E9E
:1476C40028822BE130E000270E9497030E94D00321960895C0
:1476D80021974090CA025090CB022090C8023090C9022092E6
:1476EC00840328822AE130E000270E9497030E94D00388E0FE
:1477000090E04090CA025090CB022090C8023090C9028A939A
:14771400810192010E941B3E1093D1020093D0023093D302DE
:147728002093D2021801290120928403288229E130E000275F
:14773C000E9497030E94D00388E090E04090D2025090D30257
:147750002090D0023090D1028A93810192010E941B3E009350
:147764008403202E288228E130E000270E9497030E94D003A1
:14777800219608950E94AB3D5801A89500EF19E422E030E08B
:14778C006BD005C0C501885E93405C0196D087EE93E08A1520
:1477A0009B05B0F39DD0A89505C0C501845690405C0189D0FD
:1477B40083E690E08A159B05B0F390D0A89504C0C5010A973E
:1477C8005C017DD089E090E08A159B05B8F384D0A89504C0EB
:1477DC00C50101975C0171D0AA20D1F7BB20C1F700E711E19F
:1477F00021E030E037D09698A89508E813E120E030E030D00E
:14780400969AA89500E117E220E030E029D09698A89508E8C5
:1478180013E120E030E022D0969AA89500E711E121E030E00F
:14782C001BD00E94993D08950E94AB3DA02E2A2C209432B202
:14784000322032BA00E516E420E030E00BD022B22A2822BA2A
:1478540000E516E420E030E003D00E94993D08950E94913CDA
:14786800249780E090E0A0E0B0E0FE0180839183A283B38300
:14787C0013C0A89581E090E0A0E0B0E0FE01208031804280F5
:147890005380280E391E4A1E5B1EFE012082318242825382B6
:1478A400FE012480358046805780FE016080718082809380F6
:1478B8006214730484049504F4F228960895969800E516E460
:1478CC0020E030E0C9DF969A00E516E420E030E0C3DF089592
:1478E00008EF14E221E030E0BDDF969808E813E120E030E0D8
:1478F400B7DF969A08EF14E221E030E0B1DF089517FF0895DC
:14790800109501951F4F0895A02FB12FE22FF32F01900D9213
:14791C000020E1F708953A932A931A930A9308956894DA92E9
:14793000D12E04C0E894DA92D12ED32617FF04C0109500958C
:147944000F5F1F4F37FF04C0309520952F5F3F4F0E94B73C2E
:14795800D7FE04C0109500950F5F1F4FD9900895689401C0A9
:14796C00E894EA92FA928A93EE24FF2480E1000F111FEE1C87
:14798000FF1CE216F30618F0E21AF30A03958A95A1F716F48D
:147994000E2D1F2D8991F990E9900895E89401C068942FD067
:1479A800CC2408C0E89401C0689429D037FD53D0B7FD5AD0AC
:1479BC00772488249924AA24BB2441D0C1F044D0B1F0E8E2C5
:1479D000000F111F221F331F771C881C991CAA1CBB1C8816AA
:1479E4009906AA06BB0628F0881A990AAA0ABB0A0395EA9592
:1479F80059F726F4082D192D2A2D3B2D13C07A928A929A92B0
:147A0C00AA92BA92CA92EA938A939A93AA93BA938B859C8500
:147A2000AD85BE85C32E0EF0CB260895C7FC17D0B991A99132
:147A340099918991E991C990B990A9909990899079902496A0
:147A48000895E02FE12BE22BE32B0895E82FE92BEA2BEB2B64
:147A5C00089500951095209530950F5F1F4F2F4F3F4F089540
:147A700080959095A095B0958F5F9F4FAF4FBF4F08956894CD
:147A840001C0E8942A93FA92EA92FF24EE2420E1000FFF1C8C
:147A9800EE1CE11610F0E11A03952A95B9F70EF40E2DE99021
:147AAC00F990299108950A921A928A939A93029FC001129F41
:147AC000900D039F900D8C01999189911990099008950E9484
:147AD400B63D7F920E94CF3D39F177240E94D53D19F48C01D9
:147AE8009D0120C0089FB02CA12C289F902C812C189FA00C29
:147AFC00911C871C099FA00C911C871C199F900C811C0A9FE8
:147B1000900C811C389F800C299F800C1A9F800C0B9F800CF6
:147B24000B2D1A2D292D382D7F900C94C43DE4E0A990B9901D
:147B3800E2FD0895C990D990E3FD0895E990F9900895E8E017
:147B4C000C949A3DEE270C949A3DBA92AA920895DA92CA9235
:147B60000C94AB3DFA92EA920C94AE3D8A929A92AA92BA9226
:147B7400EA938A939A93AA93BA9389859A85AB85BC85089571
:147B8800B991A99199918991E991B990A99099908990249629
:147B9C000895EE27E02BE12BE22BE32B0895EE27E82BE92B18
:147BB000EA2BEB2B0895FA93EA93BA93AA939A938A933A934E
:147BC4002A931A930A939A928A927A926A925A924A923A92C2
:147BD8002A921A920A920FB60A92089509900FBE09901990EF
:147BEC002990399049905990699079908990999009911991B9
:147C00002991399189919991A991B991E991F99108950F92E2
:147C14000990002031F0000F111F221F331F0A94F8CF0F90AC
:147C28000895112319F0000F1A95FBCF08950F9209900020EF
:147C3C0031F036952795179507950A94F8CF0F9008950A9207
:147C50001A92002411240030010741F01695079510F4020E57
:147C6400131E220F331FF5CF002D112D199009900895AA930D
:147C7800BA93EA93FA930A92AF81B885ED81FE810030010773
:147C8C0031F0C8950D92319601501040F7CF0990F991E991FC
:147CA000B991A99124960895AA93BA93EA93FA930A92AF8195
:147CB400B885ED81FE810030010729F001900D920150104070
:147CC800F8CF0990F991E991B991A991249608950E94AB3DDF
:147CDC00A02E2090EF043090F004222011F4332029F08A2D05
:147CF0008A3011F40DE0F0DF5D9BFECFACB80A2D11270E94CB
:147D0400993D08950E94913C0E94B23D622E732EA297ECA4FE
:147D1800FDA4862D972D8030E0E09E074CF4CC24C39480958E
:147D2C0090958F5F9F4F682E792E01C0CC24222429A28C2F88
:147D40009D2F8196A82EB92E8A2D9B2D0197282E392EA82EE5
:147D5400B92E2E2D3F2D062D172D0E94963CE02FF12F84E5EA
:147D680092E0E80FF91F4080E22DF32D40822E2D3F2D062DDB
:147D7C00172D0E949A3C602E712E6620F9F67720E9F6CC2033
:147D900059F08A2D9B2D0197282E392EA82EB92E8DE2E22D87
:147DA400F32D80832A2D3B2D08A519A50E94883CA2960E943E
:147DB800A83D2496089510937A020093790208952091790285
:147DCC0030917A020DE61EE40E94273E802F912F875C9F4C2D
:107DE0009F7790937A0280937902082F192F089534
:00000001FF
